:100000000C9446020C9463020C9463020C946302F9
:100010000C9463020C9463020C9463020C946302CC
:100020000C9463020C94FA0B0C9463020C9463021C
:100030000C9466160C9463020C9463020C943216B2
:100040000C9463020C9463020C94260B0C946302D0
:100050000C9439040C9463020C9403040C94630212
:100060000C94CF0C0C9463020C9469150C946302ED
:100070000C941D3B0C9463020C9463020A0A0D005D
:100080004E65757472616C0048656164696E67489D
:100090006F6C64000A0D436F6E74726F6C3A2000CF
:1000A0004F4B0A0D000A0D43616C696272617469FD
:1000B0006E67206169722070726573737572652056
:1000C00073656E736F722E2E000A0D414343206ECE
:1000D0006F742063616C6962726174656421000AE7
:1000E0000D3D3D3D3D3D3D3D3D3D3D3D3D3D3D3D70
:1000F0003D3D3D3D3D3D3D3D3D3D3D3D3D3D3D006D
:100100000A0D466C69676874436F6E74726F6C0A8F
:100110000D48617264776172653A25642E25640A20
:100120000D536F6674776172653A5625642E2564A7
:10013000256320002E0048693A2534692020436653
:100140003A253469200047733A25346920205961E3
:100150003A25346920004E693A2534692020526FCF
:100160003A253469200045787465726E436F6E7469
:10017000726F6C20200052616E67653A2533692DDD
:1001800025336900506F736974696F6E3A202533A7
:100190006900536574706F696E742020253369009F
:1001A000536572766F202000506F343A20253369F2
:1001B00020506F383A2025336900506F333A20259C
:1001C000336920506F373A2025336900506F323A37
:1001D0002025336920506F363A2025336900506F4F
:1001E000313A2025336920506F353A202533690094
:1001F0004F6666436F757273653A2025356900480E
:10020000656164696E673A20202025356900436F77
:10021000757273653A2020202025356900436F6D83
:1002200070617373202020202020200052432D4C29
:100230006576656C3A2025356900566F6C74616788
:10024000653A20202535690048656967687420256E
:10025000346920282533692900526F6C6C202020D6
:10026000253469202825336929004E69636B2020D5
:1002700025346920282533692900414343202D2056
:1002800053656E736F7200596177202020253469A1
:1002900020282533692900526F6C6C202025346991
:1002A000202825336929004E69636B202534692095
:1002B00028253369290059617720202025346920B9
:1002C000282533692900526F6C6C20202534692061
:1002D0002825336929004E69636B2025346920285D
:1002E00025336929004779726F202D2053656E737D
:1002F0006F720050333A253469202050343A253447
:1003000069200050313A253469202050323A253492
:1003100069200047733A253469202059613A253411
:100320006920004E693A2534692020526F3A2534FD
:1003300069200043373A253469202043383A253470
:1003400069200043353A253469202043363A253464
:1003500069200043333A253469202043343A253458
:1003600069200043313A253469202043323A25344C
:1003700069200048656164696E673A202020253550
:100380006900526F6C6C3A202020202020253569AE
:10039000004E69636B3A20202020202535690041FA
:1003A000747469747564650048656967687420438E
:1003B0006F6E74726F6C004E6F20004F66667365CF
:1003C00074202020203A253569004169722050723E
:1003D0006573732E3A2535690053657420506F6933
:1003E0006E743A20253569004865696768743A205B
:1003F0002020202535690028632920486F6C676517
:100400007220427573730053657474696E673A2085
:100410002564200048573A5625642E2564205357FA
:100420003A25642E25642563002B204D696B726F7D
:100430004B6F70746572202B005B25695D005B2536
:10044000695D000A0D5573696E6720506172616DB8
:100450006574657220536574202564000A0D496E29
:1004600069742E20454550524F4D3A2047656E65C0
:10047000726174696E672044656661756C742D5095
:100480006172616D657465722E2E2E0011241FBE7F
:10049000CFEFD0E1DEBFCDBF14E0A0E0B1E0E4ECEF
:1004A000FFE702C005900D92A23BB107D9F718E013
:1004B000A2EBB4E001C01D92AB3AB107E1F70E9494
:1004C00065020C94E13F0C940000CF93DF93F89405
:1004D00014B815B8189B02C08BE001C08AE0809365
:1004E000000184B1836084B9209100012A3011F4A5
:1004F000289A01C02898299884B7877F84BF809163
:1005000060008861809360001092600080ED97E049
:100510009093CE048093CD041092640710926307E9
:1005200010926D0510926C0510926B0510926A0581
:1005300010926905109268052A3011F4289801C0BC
:10054000289A0E94B9140E94F10A0E94D70B0E94B7
:10055000D405809100018B3011F40E94C03A0E94B2
:10056000FE150E94B20C0E9412157894109261063A
:1005700085E48093620687E0809363062091000102
:10058000822F6AE00E94123F492F50E0822F0E9482
:10059000123F90E02BE630E03F932F9325E430E0CC
:1005A0003F932F931F921F925F934F939F938F932D
:1005B00080E091E09F938F931F920E944D088FEDF2
:1005C00090E09F938F931F920E944D08299A0E945A
:1005D000093A84E00E9409382DB73EB7205F3F4FAB
:1005E0000FB6F8943EBF0FBE2DBF8050944050F020
:1005F00089EC90E09F938F931F920E944D080F907B
:100600000F900F9084EF91E00E948A0BEC01CE01D5
:100610000E94930B8823D9F38091CF0780FF20C0DD
:1006200085EA90E09F938F931F920E944D0888EE79
:1006300093E00E948A0BEC010E94AE0F0F900F9086
:100640000F90CE010E94930B8823D9F380EA90E0AB
:100650009F938F931F920E944D080F900F900F90C1
:100660000E944E20809100018A3011F4289801C028
:10067000289A80ED97E09093CE048093CD0485E591
:1006800080936B0684E990E09F938F931F920E9462
:100690004D088091CF070F900F900F9082FF03C0FD
:1006A00088E890E002C080E890E09F938F931F92CB
:1006B0000E944D080F900F900F908CE790E09F9351
:1006C0008F931F920E944D080E94EE0F80ED97E0DD
:1006D00090936D0380936C030F900F900F90809117
:1006E000CA048823E1F31092CA040E94F8210E94F0
:1006F0001720209100012A3011F4289801C0289A6F
:1007000080910301882321F081508093030112C05E
:100710001092BE041092BF041092750610927905D3
:100720001092780510927B0510927A0510927D0543
:1007300010927C0580916C0390916D03892B01F5DB
:1007400085E090E090936D0380936C030E943915CF
:1007500080910403909105038F5F9F4FF9F480917E
:1007600054058823D9F080E197E29093CE048093DA
:10077000CD0480E890E090930503809304030EC0BD
:1007800080916C0390916D03019790936D0380931A
:100790006C032A3011F4289801C0289A8091CA0469
:1007A000882321F080915405882311F40E943B0690
:1007B0000E94E306CE010E94930B882309F48FCF99
:1007C00020910803309109038091DF0790E02817FA
:1007D00039079CF480910403909105038F5F9F4F2C
:1007E00061F480E797E19093CE048093CD0480E09C
:1007F00093E0909305038093040384E190E00E94CA
:100800008A0BEC016CCF1F920F920FB60F9211243E
:100810008F939F93EF93FF93809102018823E1F4DC
:100820008091C6049091C70401969093C704809369
:10083000C604FC01E854F94FE081ED3019F0863927
:10084000910539F41092C7041092C60481E0809398
:100850000201E093C60004C01092C7041092C604BF
:10086000FF91EF919F918F910F900FBE0F901F906E
:1008700018951F920F920FB60F9211242F933F934A
:100880004F935F936F937F938F939F93AF93BF9398
:10089000CF93DF93EF93FF937091C6008091B804DC
:1008A000882309F06DC06091C304662371F473322C
:1008B00079F47093C90581E08093C30483E290E0EA
:1008C0009093C5048093C4045BC0663908F054C09B
:1008D000A62FB0E02091C4043091C5047D3069F0AA
:1008E000A753BA4F7C936F5F6093C304270F311DEA
:1008F0003093C5042093C40443C0FD01E953FA4F6B
:100900009081ED01C853DA4F8881A901491B510933
:10091000481B51095F705093C5044093C404208163
:10092000CA0136E0969587953A95E1F7835C821780
:10093000F1F49881842F8F73835C8917C1F481E06F
:100940008093B8046093B904A753BA4F7C93809105
:10095000CB05823571F488E190E02CE00FB6F89475
:10096000A895809360000FBE2093600002C0109293
:10097000B8041092C30404C01092C3041092B804C7
:10098000FF91EF91DF91CF91BF91AF919F918F91A7
:100990007F916F915F914F913F912F910F900FBE7B
:1009A0000F901F901895DC0120E030E040E050E00F
:1009B00008C0FA01E854F94F8081280F311D4F5FBC
:1009C0005F4F4A175B07A9F73F70C90146E096954C
:1009D00087954A95E1F7835CFD01E854F94F8083E0
:1009E00011962F73235CFD01E854F94F2083A7541F
:1009F000B94F8DE08C93109202018091B8068093DC
:100A0000C60008951F93CF93DF93EA01722F93E2FC
:100A10009093B8066093B9068093BA06A3E0B0E05D
:100A200060E04FC0FE01E60FF11D90816F5F7150D5
:100A300019F410E040E00FC0FE01E60FF11D408107
:100A40006F5F715011F410E006C0FE01E60FF11D5A
:100A500010816F5F7150892F86958695835CFD01AB
:100A6000E854F94F808350E09A0184E03695279549
:100A70008A95E1F7892F90E083709070F4E0880FF9
:100A8000991FFA95E1F7282B235CFD01E754F94FF4
:100A90002083812F82958695869583704F70507044
:100AA000440F551F440F551F842B835CFD01E654F2
:100AB000F94F80831F73135CFD01E554F94F1083D8
:100AC0001496772309F0AECFCD010E94D304DF91B5
:100AD000CF911F9108951F93CF93DF93EC0170E0A6
:100AE000A22FB0E0129748C0E42FF0E0E753FA4F8E
:100AF00030814F5FE42FF0E0E753FA4F50814F5FB2
:100B0000E42FF0E0E753FA4F10814F5FE42FF0E05D
:100B1000E753FA4F20814F5F842F90E0A817B90761
:100B200074F15D53FE01E70FF11D852F82958F70E3
:100B30003D53330F330F382B3083613001F1912F48
:100B40009D537F5FFE01E70FF11D71505295507F5D
:100B5000892F86958695582B508363506F3F79F087
:100B60007E5FFE01E70FF11D9295990F990F907C22
:100B70002D53922B90837F5F662309F0B5CFDF91D1
:100B8000CF911F9108951F93182F8A3019F48DE08B
:100B90000E94C3058091C00085FFFCCF1093C60062
:100BA00080E090E01F9108951F931FB7F894809103
:100BB000C1008F778093C1008091C1008F7B8093AB
:100BC000C100589A5098599A519A1092C5008AE2D9
:100BD0008093C4008091C00082608093C00088E14F
:100BE0008093C1008091C2008F778093C200809172
:100BF000C2008F7B8093C2008091C2008F7D809362
:100C0000C2008091C2008F7E8093C2008091C2009A
:100C1000877F8093C2008091C1008B7F8093C10049
:100C20008091C20084608093C2008091C200826083
:100C30008093C20002C08091C6008091C00087FDF1
:100C4000FACF8091C10080688093C1008091C1007B
:100C500080648093C1001092B80481E08093020107
:100C600088EC90E00E948A0B9093600680935F0668
:100C70001FBF1F91089580910201882309F4A2C02B
:100C80008091B304882371F080910201882351F090
:100C90006091C2042BE04BE656E087E40E94020517
:100CA0001092B30480915F06909160060E94930BAE
:100CB000882321F48091B5048823B1F0809102014A
:100CC000882391F06091C20422E446E756E084E470
:100CD0000E9402051092B5048AEF90E00E948A0BF0
:100CE0009093600680935F06609101016F3F89F0E9
:100CF000462F50E094E0440F551F9A95E1F74C5F62
:100D00005E4F605D20E181E40E9402058FEF8093D9
:100D1000010190914E079923A1F08091020188234F
:100D200081F083E28093B8069093B9068DE08093BA
:100D3000BA061092020110924E078091B806809375
:100D4000C6008091B404882359F180910201882360
:100D500039F10E94F70F1092B4043091B704932F29
:100D60009F5F9093B704943021F08091B60488235C
:100D700059F02EE14FE557E060E084E30E94020560
:100D80008FEF8093B7040CC044E1949FA00111241D
:100D9000465E5C4F24E160E0832F8F5C0E94020579
:100DA0008091B204882371F080910201882351F070
:100DB0006091C2042AE041E656E086E50E94020501
:100DC0001092B20408951F93CF93DF93CDB7DEB78F
:100DD00022970FB6F894DEBF0FBECDBF8091B80446
:100DE000882309F4F7C08091CB058B3609F47EC0C7
:100DF0008C3688F48336E1F1843630F48136C1F0E4
:100E0000823609F0E5C020C0873609F480C08836F4
:100E100009F0DEC047C0813709F47DC0813708F48E
:100E2000A4C0843709F459C0863709F0D1C06BC01B
:100E30002091B90443E062E0CE0101960E946B0567
:100E40008981809301012AC02091B90443E06BE0BD
:100E50008BE696E00E946B058091F00490916D0600
:100E6000892B8093F0048091740680934E07B0C064
:100E70002091B90443E06BE08BE696E00E946B059D
:100E80008091F00490916D06892B8093F0048091FD
:100E9000740680934E0781E08093B5048FEF8093B2
:100EA000030196C02091B90443E062E0CE010196AF
:100EB0000E946B058091F0049981892B8093F00446
:100EC0008A818F3F21F481E08093B60402C01092A2
:100ED000B60481E08093B4047BC02091B90443E060
:100EE00064E08AEB94E00E946B05D8CF2091B904AE
:100EF00043E064E08EEB94E00E946B058091C104B6
:100F000080934E07CBCF81E08093B20461C081E033
:100F10008093B3045DC02091B90443E062E0CE0148
:100F200001960E946B05809102018823E1F389817B
:100F30008F3F71F0863010F085E0898389810E94AF
:100F400037386091C204898126E447EC57E009C034
:100F50001091C20482E00E94F83726E447EC57E083
:100F6000612F855B0E94020533C02091B90443E0E4
:100F700066E487EC97E00E946B058091CB058B5669
:100F80000E9422386091F20770E080E090E024EC4B
:100F900039E040E050E00E94F33E609374037093A8
:100FA000750380937603909377036091F30770E065
:100FB00080E090E00E94F33E6093780370937903A1
:100FC00080937A0390937B030E94FA390E94B321A5
:100FD0001092B80422960FB6F894DEBF0FBECDBFB4
:100FE000DF91CF911F910895982F80914F07813005
:100FF00069F48091EF04E82FF0E0E65EFC4F908307
:101000008F5F8093EF0421E030E005C0892F0E94BC
:10101000C305282F30E0C90108951F93182F04C07D
:1010200080E30E94F40711501116D4F31F91089524
:101030001F93182F04C080E20E94F407115011166C
:10104000D4F31F9108950F931F93CF93DF938C01D7
:10105000EB0108C0F8010F5F1F4FE4918E2F0E9433
:10106000F40721972097B1F7DF91CF911F910F914E
:1010700008950F931F93CF93DF938C01EB0106C06C
:10108000F80181918F010E94F40721972097C1F701
:10109000DF91CF911F910F9108952F923F924F9220
:1010A0005F926F927F928F929F92AF92BF92CF92F8
:1010B000DF92EF92FF920F931F93CF93DF93CDB701
:1010C000DEB7E5970FB6F894DEBF0FBECDBF2B9607
:1010D0008FAD2B9780934F07CE01835B9F4F9B83F0
:1010E0008A832D964EAC5FAC2D971EA61FA618AA1C
:1010F00019AA9E01225D3F4F3DAB2CAB820102C07D
:101100000F5F1F4FF801F490FF2019F0F5E2FF1672
:10111000B9F7B8016419750919F0C2010E942308D2
:10112000FF2009F445C228010894411C511C198272
:10113000AA81BB8133241BAA2FEF2AABF2010894AA
:10114000411C511CB490632D70E06170707035E7E4
:10115000B31621F08B2D80628837C9F461157105B3
:1011600059F02D913D914D915C9113972EA73FA77A
:1011700048AB59AB14960BC08D919C9111979C0173
:1011800040E050E02EA73FA748AB59AB129630E2A3
:10119000B31621F48981882389F61CC043E2B41672
:1011A00011F458E055C08AE2B81621F09DE2B91654
:1011B00071F408C0FD011296E081EBABE7FFBECFF2
:1011C000E195EBABE0E13E2AFFED3F22B7CF2BE20A
:1011D000B21611F4B982B2CF3EE2B31699F5F2011C
:1011E0000894411C511C84918A3221F0B82E20E0D1
:1011F00030E01DC0FD0112964081518157FF02C0B1
:101200004FEF5FEF4AAB9ACFC90153E0880F991FA8
:101210005A95E1F7220F331F280F391F2B0D311D6F
:1012200020533040F2010894411C511CB4908B2D86
:1012300080538A3048F3A90137FF02C04FEF5FEFB8
:101240004AAB85CF40E3B41629F434FC77CF50E2A3
:10125000352A74CF8B2D81538930D8F420E030E0CB
:10126000C90103E0880F991F0A95E1F7220F331F88
:10127000280F391F2B0D311D20533040F2010894E7
:10128000411C511CB4908B2D80538A3048F32BABFA
:101290005ECF88E6B81619F494E0392A4FCFECE611
:1012A000BE1619F4F1E03F2A49CFBB83AA8323E697
:1012B000B21639F41296BB83AA8312978C918E834F
:1012C00022C134E4B31639F044E6B41631F059E6DD
:1012D000B516A9F502C081E0382A30FE08C0149680
:1012E000BB83AA835E914E913E912E910AC01296C5
:1012F000BB83AA839E918E919C01442737FD409524
:10130000542F2EA73FA748AB59AB8EA59FA5A8A9E0
:10131000B9A9BB238CF42EA53FA548A959A950957E
:101320004095309521953F4F4F4F5F4F2EA73FA7D8
:1013300048AB59AB8DE28983BAE02B2E80C03FE4E5
:10134000B31621F04FE6B41631F402C051E0352A4D
:10135000A8E02A2E73C080E7B81689F41296BB83E2
:10136000AA839E918E919C0140E050E02EA73FA75A
:1013700048AB59AB30E4332AF8E7BF2E5DC043E7F2
:10138000B416D1F51296BB83AA83DE90CE90C11419
:10139000D10489F488E28E838EE68F8385E788877F
:1013A0008CE689878A8789E28B871C86E6E0CE2EC9
:1013B000D12CCC0EDD1E5AA957FD14C0452F552740
:1013C00047FD509560E070E0C6010E94CB3C00975D
:1013D00011F4FAA80EC0F82EFC188AA98F154CF447
:1013E000F82E07C0F60101900020E9F73197FE2E94
:1013F000FC18198240E090C095E5B91621F0A5E7E8
:10140000BA1631F402C0B1E03B2A7AE0272E16C0AA
:10141000E8E5BE1621F0F8E7BF1609F070C033FE0C
:101420000BC02EA53FA548A959A921153105410595
:10143000510511F030E4332A60E1262E19824AA9C1
:1014400047FD02C05FED35228EA59FA5A8A9B9A9C9
:101450000097A105B10549F49AA9992331F45EE2F8
:10146000C52ED12CCC0EDD1E46C06EA47FA488A84C
:1014700099A84EE2C42ED12CCC0EDD1EE22CFF2406
:1014800000E010E06EA57FA588A999A9A8019701A1
:101490000E94453F6A3020F430E3A32EA60E08C018
:1014A00027E5A22EA60EA8E5BA1611F4BFEDAB22D1
:1014B000F601A2926F016EA57FA588A999A9A8013E
:1014C00097010E94453F2EA73FA748AB59AB6E142A
:1014D0007F048006910618F039014A01D3CFF8E065
:1014E0002F1649F433FE07C020E3A21621F080E353
:1014F000D6018E936D01FCA8FC184AA90DC0BB2033
:1015000009F456C0BE82198296E0C92ED12CCC0EA9
:10151000DD1E40E0FF24F394E42EEF18E7FCEE24F8
:101520008981882319F08F2D8F5F06C036FC02C099
:101530008F2D02C08F2D8E5FA82EAE0C032D10E0D4
:1015400080E3882E912C802291228114910421F431
:101550008BA98A190E9418088981882329F061E0E3
:1015600070E0CE01019609C006FF09C080E38C83BC
:10157000BD8262E070E0CE0104960E943908B0E2BC
:101580008B16910421F48BA98A190E940D088E2DC7
:101590000E940D086F2D772767FD7095C6010E9488
:1015A000390804FFABCD8BA98A190E941808A6CD73
:1015B000E5960FB6F894DEBF0FBECDBFDF91CF9199
:1015C0001F910F91FF90EF90DF90CF90BF90AF9061
:1015D0009F908F907F906F905F904F903F902F9053
:1015E00008952FB7F894909100019A3019F4529A07
:1015F0005A9802C03F9A479884B1886184B985B1EE
:10160000877E85B99A3019F4529A5A9802C03F9A47
:10161000479884B58F7A84BD84B5836A84BD85B5C7
:10162000877385BD85B5887F826085BD17BC88E7D7
:1016300088BD16BC80916E00897F80936E0080917A
:101640006E00816080936E002FBF08951F920F92ED
:101650000FB60F9211242F933F938F939F938091F6
:10166000CF0481508093CF048F3FB9F489E08093F9
:10167000CF04809106038F5F8170809306038823D7
:1016800019F481E08093CA048091C8049091C90440
:1016900001969093C9048093C8048091CD049091E1
:1016A000CE04892BB1F08091CD049091CE040197A6
:1016B0009093CE048093CD042091CD043091CE043C
:1016C000809104039091050382239323892BA1F435
:1016D00006C08FEF9FEF90930503809304038091E2
:1016E00000018A3039F404C05A9A0BC0479A09C0E5
:1016F0005A9807C0479805C0809100018A30B1F719
:10170000F3CF9F918F913F912F910F900FBE0F902C
:101710001F9018952091C8043091C9042F5F3F4F46
:10172000820F931F08952091C8043091C904821B31
:10173000930B892F99278695807490E00895AC01CA
:101740002091C8043091C9042F5F3F4F05C080919C
:101750007A00886C80937A008091C8049091C904C3
:10176000B901681B790BCB01840F951F80709078AD
:10177000892F99278695882351F30895AC012091EC
:10178000C8043091C9042F5F3F4F8091C8049091E5
:10179000C904B901681B790BCB01840F951F8070B8
:1017A0009078892F99278695882379F308959FB794
:1017B000F894579A5F9AE0EBF0E080818F7880830D
:1017C000808183688083E1EBF0E080818673808391
:1017D0008081866080838AE08093B3001092B2009B
:1017E000E0E7F0E080818A7F80838081826080836F
:1017F0009FBF08951F920F920FB60F921124FF9270
:101800000F931F932F933F934F935F936F937F9308
:101810008F939F93AF93BF93EF93FF9380910703B1
:101820008150809307038F3F09F082C08091B00000
:101830008093B0008091B00080688093B000809168
:10184000930390E09093D1048093D0048091FC079F
:10185000F090E90780FF23C00091D0041091D104DB
:1018600060911605709117058091180590911905E2
:1018700020E830E040E050E00E94673FCA01B90133
:101880002F2D30E040E050E00E94F33E20E032E0B7
:1018900040E050E00E94673F020F131F22C00091FA
:1018A000D0041091D10460911605709117058091B4
:1018B00018059091190520E830E040E050E00E94C2
:1018C000673FCA01B9012F2D30E040E050E00E948F
:1018D000F33E20E032E040E050E00E94673F021B10
:1018E000130B1093D1040093D0042091D0043091B5
:1018F000D1048091EA0790E02817390754F020912D
:10190000D0043091D1048091EB0790E082179307C7
:1019100024F49093D1048093D0048091D0049091CA
:10192000D1048093B3008091EC078093070306C035
:101930008091B0008F738093B0005F98FF91EF911A
:10194000BF91AF919F918F917F916F915F914F91D7
:101950003F912F911F910F91FF900F900FBE0F900D
:101960001F9018959FB7F89411B812B88FEF809315
:101970007E00ECE7F0E080818F7180838081807E43
:101980008083AAE7B0E087E28C93EBE7F0E0808108
:10199000887F80838C91886C8C939FBF08951F9261
:1019A0000F920FB60F921124EF92FF920F931F9395
:1019B0002F933F934F935F936F937F938F939F9357
:1019C000AF93BF93CF93DF93EF93FF9380917A0010
:1019D000877380937A008091ED048F5F8093ED048C
:1019E0008150853009F47EC0863090F4823009F44D
:1019F00040C0833030F48823F1F0813009F082C296
:101A00002FC0833009F441C0843009F07BC25AC032
:101A1000883009F4B2C0893038F4863009F473C0D4
:101A2000873009F06FC28CC0893009F4C3C08A3096
:101A300009F068C2DBC180917800909179009093A1
:101A4000EC048093EB0481E08093EE048091E20447
:101A50009091E30401969093E3048093E20456C2CC
:101A600080917800909179009093EA048093E90442
:101A700082C080917800909179009093E8048093DF
:101A8000E70484E08093EE0441C240910803509142
:101A9000090380917800909179009A01220F331FF9
:101AA000240F351F63E070E00E941E3F260F371F92
:101AB000369527953695279530930903209308038B
:101AC00086E0E0CF8091100590911105209178007B
:101AD00030917900821B930B9093DB048093DA049E
:101AE00087E0D0CF809178009091790020910E0509
:101AF00030910F05821B930B9093DD048093DC04DF
:101B00001092EE0403C2809100012091EB04309109
:101B1000EC048A3049F48091780090917900820F2A
:101B2000931F9695879506C08091780090917900D3
:101B3000820F931F9093D9048093D80481E0A2CFA1
:101B4000809100012091E9043091EA048A3049F43F
:101B50008091780090917900820F931F96958795D8
:101B600006C08091780090917900820F931F909326
:101B7000D7048093D60482E085CF80910001209124
:101B8000E7043091E8048A3049F48091780090911C
:101B90007900820F931F9695879506C080917800F3
:101BA00090917900820F931F9093D5048093D40471
:101BB00085E068CF6091780070917900E09012051F
:101BC000F09013050091140510911505882777FDF5
:101BD0008095982F0E94D83DA80197010E94D83C7B
:101BE0000E94A53D7093DF046093DE04E091DE0463
:101BF000F091DF048091DC049091DD04C091DA045F
:101C0000D091DB0497FF03C0909581959F4F64E0CE
:101C100070E00E94323F9B01CE01D7FF03C0909538
:101C200081959F4F64E070E00E94323F260F371F7E
:101C3000E20FF31FF093DF04E093DE048091DE04F3
:101C40009091DF0402970CF43EC0609112057091F0
:101C50001305809114059091150520E030E84BE3C1
:101C600054E40E94133E88230CF078C06091120562
:101C70007091130580911405909115052AE037EDB8
:101C800043EA5CE30E94D93C60931205709313050C
:101C900080931405909315058091560590915705F2
:101CA000845F914008F05AC060911205709113054D
:101CB00080911405909115052DEC3CEC4CEC5DE306
:101CC0000E94D93C43C08091DE049091DF048F5F75
:101CD0009F4F0CF043C060911205709113058091E5
:101CE00014059091150520E030E849E054E40E9485
:101CF000173E18169CF5609112057091130580919E
:101D00001405909115052AE037ED43EA5CE30E9443
:101D1000D83C60931205709313058093140590933B
:101D200015058091560590915705845F9140B0F458
:101D3000609112057091130580911405909115051D
:101D40002DEC3CEC4CEC5DE30E94D83C609312051A
:101D50007093130580931405909315058091780076
:101D6000909179009093D3048093D20420914605FA
:101D70003091470540914805509149058091DE0416
:101D80009091DF04AA2797FDA095BA2F820F931F89
:101D9000A41FB51F8093460590934705A09348055F
:101DA000B0934905E0904605F0904705009148053D
:101DB000109149056091460570914705809148054D
:101DC0009091490520E034E040E050E00E94673FF8
:101DD000E21AF30A040B150BE0924605F092470550
:101DE000009348051093490583E04CCEE0917800BC
:101DF000F09179008091E4049091E504E80FF91FD7
:101E0000F093E504E093E4048091E6048F5F80930F
:101E1000E604853008F476C08091780090917900CE
:101E200090930F0380930E034091E0045091E104DE
:101E300020915007309151072E1B3F0B80917E055A
:101E400090917F05281B390B8091820390E0BC01A3
:101E5000269FC001279F900D369F900D11249A0157
:101E6000A3E0220F331FAA95E1F7241B350B820F45
:101E7000931F68E070E00E94323F7093E10460932A
:101E8000E004E0900A03F0900B0300910C03109122
:101E90000D03BF01882777FD8095982FA801970132
:101EA000220F331F441F551F2E0D3F1D401F511F72
:101EB000620F731F841F951F24E030E040E050E064
:101EC0000E94673F20930A0330930B0340930C0357
:101ED00050930D03209150073091510780910A03D0
:101EE00090910B03A0910C03B0910D03281B390BAB
:101EF00030937F0520937E051092E6041092E5044E
:101F00001092E4041092EE041092ED0480917C0093
:101F1000807E9091EE04892B80937C008091ED046B
:101F2000882329F080917A00886C80937A00FF9151
:101F3000EF91DF91CF91BF91AF919F918F917F9161
:101F40006F915F914F913F912F911F910F91FF9052
:101F5000EF900F900FBE0F901F9018951F93CF9387
:101F6000DF9383E00E94F837182F853108F01A506C
:101F700017BD84E690E00E949F0B80910E03909124
:101F80000F0382559340C0F410E016C017BD82E3E2
:101F900090E00E949F0BDF93CF931F920E944D0809
:101FA00080910E0390910F030F900F900F90845823
:101FB000934030F01F5F02C0C4E3D1E01A3F30F31A
:101FC000612F83E00E940138109352078CE291E068
:101FD0000E949F0BDF91CF911F910895EAE1F3E0FA
:101FE00080E2819383E0EA36F807D1F708951F93E2
:101FF0008091F004282F30E0C90181709070682F23
:102000008823A9F08091F104882311F0815002C047
:1020100080916A038093F104EAE1F3E080E2819326
:1020200083E0EA36F807D1F78FEF8093B704A90170
:102030004270507021FF17C09091F10480916A03A3
:10204000981719F41092F10403C09F5F9093F10464
:10205000EAE1F3E080E2819393E0EA36F907D1F711
:102060008FEF8093B704662321F0452B11F0109277
:10207000F1048091F104282F30E08A3040F481E1AE
:102080008093EF043F932F938EE394E007C080E1A9
:102090008093EF043F932F9389E394E09F938F9372
:1020A00081E08F930E944D080F900F900F900F903A
:1020B0000F901091F104153009F4FBC1163090F423
:1020C000123009F4D0C0133030F4112309F111306B
:1020D00009F046C465C0133009F41BC1143009F07F
:1020E0003FC46BC1183009F411C3193038F41630ED
:1020F00009F499C2173009F033C4E3C21A3009F465
:102100009FC31A3008F440C31B3009F029C4D6C35A
:102110001092EF0489E294E09F938F9311E01F9354
:102120000E944D0884E18093EF0420910001822FEA
:102130006AE00E94123F492F50E0822F0E94123F16
:1021400090E02BE630E03F932F9325E430E03F937F
:102150002F931F921F925F934F939F938F9384E1CE
:1021600094E09F938F931F930E944D0888E2809381
:10217000EF040E94FA3990E09F938F9387E094E0F8
:102180009F938F931F930E944D088CE38093EF04DD
:1021900087EF93E09F938F931F930E944D08DCC3BA
:1021A0008091CF0780FF47C01092EF0480917E0599
:1021B00090917F059F938F9388EE93E09F938F93E9
:1021C0001F930E944D0884E18093EF048091800565
:1021D000909181059F938F9389ED93E09F938F93C7
:1021E0001F930E944D0888E28093EF0480910E03B4
:1021F00090910F039F938F938AEC93E09F938F931B
:102200001F930E944D088CE38093EF048091520746
:1022100090E09F938F938BEB93E09F938F931F930B
:102220000E944D088DB79EB744960FB6F8949EBF96
:102230000FBE8DBF9AC384E18093EF0487EB93E0D8
:102240009F938F931F930E944D0888E28093EF0421
:1022500088EA93E09F938F931F930E944D088DB758
:102260009EB70696E2CF1092EF048FE993E09F931A
:102270008F9311E01F930E944D0884E18093EF0437
:1022800060911605709117058091180590911905B8
:1022900020E034E040E050E00E94673F5F934F93BE
:1022A0003F932F9381E993E09F938F931F930E9415
:1022B0004D0888E28093EF0460911E0570911F0520
:1022C000809120059091210520E034E040E050E02D
:1022D0000E94673F5F934F933F932F9382E893E071
:1022E0009F938F931F930E944D088CE38093EF047C
:1022F00080916E0390916F039F938F9383E793E098
:102300009F938F931F930E944D088DB79EB746965B
:102310008CCF1092EF048091630790916407209115
:102320006107309162079F938F933F932F9383E6CA
:1023300093E09F938F9311E01F930E944D0884E1D7
:102340008093EF048091670790916807209165075B
:10235000309166079F938F933F932F9383E593E08C
:102360009F938F931F930E944D0888E28093EF0400
:1023700080916B0790916C072091690730916A07F3
:102380009F938F933F932F9383E493E09F938F9337
:102390001F930E944D088CE38093EF0480916F0798
:1023A0009091700720916D0730916E079F938F93E6
:1023B0003F932F9383E393E03AC21092EF04E091AE
:1023C000C807F0E0EE0FFF1FE15AF84F208131817E
:1023D000E091C707F0E0EE0FFF1FE15AF84F808150
:1023E00091813F932F939F938F9383E293E09F93E9
:1023F0008F9311E01F930E944D0884E18093EF04B6
:10240000E091CA07F0E0EE0FFF1FE15AF84F20817C
:102410003181E091C907F0E0EE0FFF1FE15AF84F5C
:10242000808191813F932F939F938F9383E193E0DA
:102430009F938F931F930E944D0888E28093EF042F
:10244000E091CC07F0E0EE0FFF1FE15AF84F20813A
:102450003181E091CB07F0E0EE0FFF1FE15AF84F1A
:10246000808191813F932F939F938F9383E093E09B
:102470009F938F931F930E944D088CE38093EF04EA
:10248000E091CE07F0E0EE0FFF1FE15AF84F2081F8
:102490003181E091CD07F0E0EE0FFF1FE15AF84FD8
:1024A000808191813F932F939F938F9383EF92E04D
:1024B000BEC11092EF0485EE92E09F938F9311E0DE
:1024C0001F930E944D080F900F900F908091000174
:1024D0008A3009F04AC084E18093EF0440910405FA
:1024E000509105058091D4049091D5042091040564
:1024F00030910505821B930B5F934F939F938F93AE
:1025000086ED92E09F938F931F930E944D0888E27F
:102510008093EF0440910605509107058091D60401
:102520009091D7042091060530910705821B930BEB
:102530005F934F939F938F9386EC92E09F938F933B
:102540001F930E944D088CE38093EF04809108054F
:10255000909109052091B4073091B5079F938F930F
:102560003F932F9386EB92E055C084E18093EF0474
:10257000809104059091050562E070E00E94323F71
:102580008091D4049091D5042091040530910505E3
:10259000821B930B7F936F939F938F9387EA92E0B5
:1025A0009F938F931F930E944D0888E28093EF04BE
:1025B000809106059091070562E070E00E94323F2D
:1025C0008091D6049091D70420910605309107059B
:1025D000821B930B7F936F939F938F9387E992E076
:1025E0009F938F931F930E944D088CE38093EF0479
:1025F000809108059091090562E070E00E94323FE9
:102600008091B4079091B5077F936F939F938F93B9
:1026100087E892E09F938F931F930E944D088DB798
:102620009EB7459602CE1092EF048AE792E09F9300
:102630008F9311E01F930E944D0884E18093EF0473
:1026400080910E0590910F052091DC043091DD04FE
:102650009F938F933F932F938AE692E09F938F935C
:102660001F930E944D0888E28093EF04809110052B
:10267000909111052091DA043091DB049F938F93A0
:102680003F932F9389E592E09F938F931F930E942E
:102690004D088CE38093EF0460911205709113054F
:1026A00080911405909115050E94A53D2091AA07DF
:1026B0003091AB077F936F933F932F9388E492E021
:1026C00046C184E18093EF0480910803909109034F
:1026D0009F938F938AE392E09F938F9311E01F93D0
:1026E0000E944D0888E28093EF048091FD04909150
:1026F000FE049F938F938CE292E09F938F931F939E
:102700000E944D088DB79EB70A968FCD1092EF04A8
:102710008DE192E09F938F9311E01F930E944D08EB
:1027200084E18093EF0480917003909171039F93F3
:102730008F938EE092E09F938F931F930E944D089A
:1027400088E28093EF0480916E0390916F039F93D2
:102750008F938FEF91E09F938F931F930E944D086B
:102760008CE38093EF0480914A0590914B059F93F1
:102770008F9380EF91E09F938F931F930E944D085A
:102780008DB79EB7429651CD1092EF0480916005AF
:102790009091610520915805309159059F938F9331
:1027A0003F932F938EED91E09F938F9311E01F93B2
:1027B0000E944D0884E18093EF048091620590911E
:1027C000630520915A0530915B059F938F933F934A
:1027D0002F938CEC91E09F938F931F930E944D0851
:1027E00088E28093EF0480916405909165052091C3
:1027F0005C0530915D059F938F933F932F938AEBF8
:1028000091E09F938F931F930E944D088CE38093D8
:10281000EF04809166059091670520915E053091E7
:102820005F059F938F933F932F9388EA91E09F9347
:102830008F931F930E944D088DB79EB74C96F5CC91
:102840001092EF0480EA91E09F938F9311E01F9321
:102850000E944D0884E18093EF048091930390E0FF
:102860009F938F9382E991E09F938F931F930E9490
:102870004D0888E28093EF048091D0049091D104B8
:102880009F938F9384E891E09F938F931F930E946F
:102890004D088CE38093EF042091EB0730E08091AA
:1028A000EA0790E03F932F939F938F9386E791E001
:1028B0009F938F931F930E944D08B4CC1092EF0406
:1028C00086E691E09F938F9311E01F930E944D083D
:1028D00084E18093EF0420916F06332727FD309524
:1028E00080916E06992787FD90953F932F939F9334
:1028F0008F9386E591E09F938F931F930E944D08DD
:1029000088E28093EF0420917006332727FD3095ED
:102910008091710690E03F932F939F938F9386E46D
:1029200091E09F938F931F930E944D088CE38093B7
:10293000EF042091750630E080917206992787FD9B
:1029400090953F932F939F938F9386E391E09F936E
:102950008F931F930E944D088DB79EB7489665CC04
:10296000115010936A031092F1041092F0041F9119
:10297000089587B18C6087B9429843980895409133
:10298000F2045091F3044431510500F14C3D5105DE
:10299000E8F42091F8043091F904C901880F991FD7
:1029A0008417950710F4429A01C042982F5F3F4F59
:1029B0003093F9042093F804215030402417350750
:1029C00030F01092F9041092F80401C0429A40913C
:1029D000F4045091F5044431510510F4439A0895DC
:1029E0004C3D5105E8F42091F6043091F704C901FB
:1029F000880F991F8417950710F4439A01C04398D4
:102A00002F5F3F4F3093F7042093F604215030405E
:102A10002417350730F01092F7041092F604089549
:102A2000439A08959FB7F8943998389A88B183608B
:102A300088B9E9EBF0E080818C7F80838AE2809323
:102A4000B8009FBF089585EA8093BC00089584E98B
:102A50008093BC0008958093BB0085E88093BC0000
:102A6000089585EC8093BC00089585E88093BC00B0
:102A70000895EF92FF920F931F938CEBE82EF12CA9
:102A800084E9F70180831092FA040BEB10E0F8015F
:102A900080818093FB041092FB0480E8F70180831F
:102AA0001092BD001092BA00F80110821092B90085
:102AB0001092B8000E94121585EAF7018083F80190
:102AC000108285E8F70180831F910F91FF90EF90AE
:102AD00008951F920F920FB60F9211248F939F9318
:102AE000EF93FF938091FA048F5F8093FA048150F3
:102AF000833009F44AC0843028F4813091F0823068
:102B0000E0F50AC0853009F447C0853008F442C0BA
:102B1000863009F05DC04CC08091FB04880F8E5A4E
:102B20001AC08091FB048F5F8093FB048150823038
:102B3000C1F0833030F4882361F0813009F055C052
:102B40000DC08430A1F0843078F0853009F04DC09C
:102B500011C08091B6078093BB0026C08091A10769
:102B6000FACF8091AC07F7CF8091BF07F4CF809167
:102B7000AD07F1CF8091C607EECF8091FB04863080
:102B800010F41092FA0485EA10C08091FC04880FBA
:102B90008D5AE1CF85EC09C0E091FC04F0E0809112
:102BA000BB00ED5AF84F808385E88093BC001DC0C0
:102BB0008091FC04E82FF0E09091BB00E95AF84FB7
:102BC00090838F5F8093FC04863010F01092FC0499
:102BD00084E98093BC001092FA048AE090E090931C
:102BE0006D0380936C031092FB04FF91EF919F9112
:102BF0008F910F900FBE0F901F9018959FB7F8946C
:102C000056985E9A8AB180638AB98BB18F7C8BB9F2
:102C1000809100018A3011F4539A5B988091800072
:102C20008C708093800080918100837E80938100EE
:102C300080918100836C80938100809182008F73EA
:102C40008093820080916F00897F80936F008091D4
:102C50006F00816280936F001092FE041092FD0459
:102C60009FBF08951F920F920FB60F9211242F93BA
:102C70003F935F936F937F938F939F93AF93BF9394
:102C80008091FF04882391F42091FD043091FE048B
:102C90008091FD049091FE0468E070E00E94323F54
:102CA000261B370B3093FE042093FD041092FF0483
:102CB000BF91AF919F918F917F916F915F913F9164
:102CC0002F910F900FBE0F901F9018951F920F928B
:102CD0000FB60F9211240F931F932F933F934F938F
:102CE0005F936F937F938F939F93AF93BF93CF9394
:102CF000DF93EF93FF9320918600309187008091BE
:102D0000000590910105281B390B80918600909158
:102D100087009093010580930005C9018D5494406C
:102D20000091020510910305835F9A4188F40430F5
:102D300011053CF010926B038091FF048F5F80932C
:102D4000FF0481E090E0909303058093020598C012
:102D50000E3011050CF094C0C9018B5F9040845B6C
:102D6000914008F072C0E901C25DD140F801EE0F58
:102D7000FF1FE15AF84F808191819E01281B390B7A
:102D8000C90137FF03C0909581959F4F069784F442
:102D90008091FD049091FE04883C91054CF4809153
:102DA000FD049091FE040A969093FE048093FD0426
:102DB000F801EE0FFF1FE15AF84F20813181C90160
:102DC000880F991F820F931F8C0F9D1F64E070E086
:102DD0000E94323F9B01CE010196861797071CF493
:102DE0002150304006C021976C177D0714F42F5FE7
:102DF0003F4F8091FD049091FE04E801CC0FDD1F50
:102E0000833C9105BCF0FE01E15AF84F808191812D
:102E1000A901481B590BCA0163E070E00E94323FD0
:102E2000CB01880F991F860F971FC358D84F9983DE
:102E3000888304C0C358D84F19821882F801EE0F56
:102E4000FF1FE15AF84F31832083F8013196F09348
:102E50000305E0930205E530F10511F45D9A06C023
:102E60005D98E630F10511F45C9A01C05C988091A0
:102E700000018A3029F4379711F45B9A01C05B98FE
:102E80008091FD049091FE04892B49F08091FD040E
:102E90009091FE0401979093FE048093FD04FF91AE
:102EA000EF91DF91CF91BF91AF919F918F917F91E2
:102EB0006F915F914F913F912F911F910F910F90C3
:102EC0000FBE0F901F9018952F923F924F925F92D6
:102ED0006F927F928F929F92AF92BF92CF92DF922A
:102EE000EF92FF920F931F93CF93DF93CDB7DEB78F
:102EF00022970FB6F894DEBF0FBECDBF80910805B4
:102F0000909109052091D8043091D904821B930B2C
:102F10009093B5078093B4078091D6049091D7041D
:102F20002091060530910705821B930B9093B30700
:102F30008093B2078091D4049091D5042091040528
:102F400030910505821B930B9093BE078093BD07BC
:102F5000E0909B07F0909C076091DC047091DD0489
:102F6000882777FD8095982F2CE030E040E050E0F6
:102F70000E94F33E0027F7FC0095102FE60EF71E87
:102F8000081F191FC801B70122E030E040E050E0FF
:102F90000E94673F30939C0720939B07E090C007F7
:102FA000F090C1076091DA047091DB04882777FD07
:102FB0008095982F2CE030E040E050E00E94F33EF6
:102FC0000027F7FC0095102FE60EF71E081F191FAB
:102FD000C801B70122E030E040E050E00E94673FC6
:102FE0003093C1072093C0072091AA073091AB0707
:102FF0006091DE047091DF04882777FD8095982F1B
:10300000442737FD4095542F620F731F841F951F6F
:1030100022E030E040E050E00E94673F3093AB0791
:103020002093AA0740913E0550913F0560914005CD
:10303000709141052091DC043091DD04C901880FB5
:10304000991F820F931F880F991F880F991FAA2716
:1030500097FDA095BA2F840F951FA61FB71F8093C9
:103060003E0590933F05A0934005B09341054091E4
:1030700042055091430560914405709145052091AA
:10308000DA043091DB04C901880F991F820F931F66
:10309000880F991F880F991FAA2797FDA095BA2F0F
:1030A000840F951FA61FB71F809342059093430579
:1030B000A0934405B09345052091DC043091DD04D4
:1030C00080914E0590914F05820F931F90934F056D
:1030D00080934E052091DA043091DB0480915005F5
:1030E00090915105820F931F909351058093500545
:1030F00080915205909153050196909353058093CA
:10310000520520913A0530913B0540913C05509184
:103110003D058091B4079091B507AA2797FDA0952A
:10312000BA2F820F931FA41FB51F80933A05909367
:103130003B05A0933C05B0933D058091B407909169
:10314000B5079C01442737FD4095542F8091B70760
:103150009091B807A091B907B091BA07280F391F0D
:103160004A1F5B1F2093B7073093B8074093B907F6
:103170005093BA07203B83E8380788E0480780E08F
:10318000580764F0205B3348484050402093B7070D
:103190003093B8074093B9075093BA078091B707A7
:1031A0009091B807A091B907B091BA07B7FF0CC0CA
:1031B00080559C47A74FBF4F8093B7079093B807A0
:1031C000A093B907B093BA07909186059A83992383
:1031D00009F08AC080918705882309F085C0809115
:1031E000CF0786FF81C06091B4077091B507209129
:1031F0002A0530912B0540912C0550912D05E0902A
:103200009503FF2400E010E0882777FD8095982F34
:103210000E94F33E20E038E040E050E00E94673F2B
:10322000CA01B901A80197010E94F33E20E030E1F4
:1032300040E050E00E94673F59016A012093C505B4
:103240003093C6054093C7055093C8056091B407F5
:103250007091B507209132053091330540913405C6
:1032600050913505882777FD8095982F0E94F33E71
:1032700020E038E040E050E00E94673FCA01B90119
:10328000A80197010E94F33E20E030E140E050E0C9
:103290000E94673F2093C1053093C2054093C30548
:1032A0005093C405D601C501D7FE07C0B095A095BF
:1032B000909581959F4FAF4FBF4F81389105A105E4
:1032C000B10574F457FF07C050954095309521958E
:1032D0003F4F4F4F5F4F2138310541055105A4F055
:1032E00081E080934D0510C01092C1051092C20577
:1032F0001092C3051092C4051092C5051092C60520
:103300001092C7051092C8058091B2079091B3073B
:103310002090C5053090C6054090C7055090C8055F
:10332000820D931D9093B3078093B2070091B2076B
:103330001091B307A090C105B090C205C090C3051D
:10334000D090C40580919603682E77248824992410
:10335000C401B301A60195010E94F33E20E032E0D2
:1033600040E050E00E94673F020F131F1093B30725
:103370000093B2072091360530913705409138050A
:10338000509139058091B2079091B307AA2797FD14
:10339000A095BA2F820F931FA41FB51F80933605E7
:1033A00090933705A0933805B093390540913205C5
:1033B0005091330560913405709135058091B207C5
:1033C0009091B3072091820530918305821B930B66
:1033D000AA2797FDA095BA2F840F951FA61FB71F88
:1033E0008093320590933305A0933405B09335054F
:1033F0008091320590913305A0913405B091350547
:10340000E0907803F090790300917A0310917B03A8
:10341000E816F9060A071B0704F580E197E2A0E029
:10342000B0E08E199F09A00BB10B809332059093E9
:103430003305A0933405B093350580913205909102
:103440003305A0913405B0913505809336059093EE
:103450003705A0933805B093390520913205309196
:103460003305409134055091350588279927DC01B3
:103470008E199F09A00BB10B281739074A075B0764
:1034800004F580EF98EDAFEFBFEFE80EF91E0A1FCD
:103490001B1FE0923205F092330500933405109320
:1034A00035058091320590913305A0913405B09196
:1034B00035058093360590933705A0933805B09372
:1034C00039058091D6049091D7040F9734F488E1A0
:1034D0009CEF9093B3078093B2078091D6049091AC
:1034E000D704079734F480E398EF9093B307809361
:1034F000B2079091000199839A30A9F48091D60483
:103500009091D704835F934034F088EE93E09093DA
:10351000B3078093B2078091D6049091D7048A5F55
:103520009340DCF014C08091D6049091D704855E5E
:10353000974034F088EE93E09093B3078093B207FE
:103540008091D6049091D704835F974034F080ED4A
:1035500097E09093B3078093B2078091BD07909155
:10356000BE078A199B099093BE078093BD070091FF
:10357000BD071091BE07C401B301A20191010E94D1
:10358000F33E20E032E040E050E00E94673F021B43
:10359000130B1093BE070093BD0720912E053091A9
:1035A0002F0540913005509131058091BD079091D4
:1035B000BE07AA2797FDA095BA2F820F931FA41FBD
:1035C000B51F80932E0590932F05A0933005B093DF
:1035D000310540912A0550912B0560912C05709181
:1035E0002D058091BD079091BE07209184053091F3
:1035F0008505821B930BAA2797FDA095BA2F840FF0
:10360000951FA61FB71F80932A0590932B05A093A3
:103610002C05B0932D0580912A0590912B05A09142
:103620002C05B0912D05E0907403F0907503009186
:10363000760310917703E816F9060A071B0704F5CD
:1036400088EA91E6A0E0B0E08E199F09A00BB10BCB
:1036500080932A0590932B05A0932C05B0932D05FC
:1036600080912A0590912B05A0912C05B0912D05F4
:1036700080932E0590932F05A0933005B0933105CC
:1036800020912A0530912B0540912C0550912D0554
:1036900088279927DC018E199F09A00BB10B2817E9
:1036A00039074A075B0704F588E59EE9AFEFBFEFEE
:1036B000E80EF91E0A1F1B1FE0922A05F0922B0547
:1036C00000932C0510932D0580912A0590912B05D0
:1036D000A0912C05B0912D0580932E0590932F0578
:1036E000A0933005B09331058091D4049091D50416
:1036F0000F9734F488E19CEF9093BE078093BD0749
:103700008091D4049091D504079734F480E398EF26
:103710009093BE078093BD0799819A30A9F4809158
:10372000D4049091D504835F934034F088EE93E005
:103730009093BE078093BD078091D4049091D504E7
:103740008A5F9340DCF014C08091D4049091D5043A
:10375000855E974034F088EE93E09093BE078093A7
:10376000BD078091D4049091D504835F974034F0D5
:1037700080ED97E09093BE078093BD0780917A001B
:10378000886C80937A0080913A0590913B05A091D6
:103790003C05B0913D058093260590932705A093A5
:1037A0002805B093290580912A0590912B05A091B9
:1037B0002C05B0912D058093160590931705A093C5
:1037C0001805B09319058091320590913305A091A9
:1037D0003405B091350580931E0590931F05A09385
:1037E0002005B093210580912E0590912F05A09181
:1037F0003005B091310580931A0590931B05A09375
:103800001C05B0931D058091360590913705A09158
:103810003805B09139058093220590932305A09334
:103820002405B09325058091CF0787FF63C02A81C7
:10383000222309F05FC080918705882309F05AC0D0
:103840008091BD079091BE07893C91055CF0209165
:10385000BD073091BE078091BD079091BE072052F1
:10386000334011C08091BD079091BE0788539F4F90
:10387000A4F42091BD073091BE078091BD079091BF
:10388000BE07205E3C4F880F991F880F991F280F95
:10389000391F3093BE072093BD078091B2079091E6
:1038A000B307893C91055CF02091B2073091B307D2
:1038B0008091B2079091B3072052334011C080919C
:1038C000B2079091B30788539F4FA4F42091B20799
:1038D0003091B3078091B2079091B307205E3C4FBF
:1038E000880F991F880F991F280F391F3093B3072E
:1038F0002093B20722960FB6F894DEBF0FBECDBF5D
:10390000DF91CF911F910F91FF90EF90DF90CF90BB
:10391000BF90AF909F908F907F906F905F904F90EF
:103920003F902F9008950F931F930AE710E0F8013E
:103930008081877380838091D4049091D504909383
:10394000BE078093BD078091D6049091D7049093D1
:10395000B3078093B2078091D8049091D9049093D3
:10396000B5078093B4076091DC047091DD0488276B
:1039700077FD8095982F2CE030E040E050E00E94E9
:10398000F33E70939C0760939B076091DA047091FB
:10399000DB04882777FD8095982F0E94F33E709373
:1039A000C1076093C0078091DE049091DF0490937B
:1039B000AB078093AA07F8018081886C80836091AF
:1039C000F20770E080E090E024EC39E040E050E065
:1039D0000E94F33E609374037093750380937603A3
:1039E000909377036091F30770E080E090E00E948D
:1039F000F33E609378037093790380937A039093F6
:103A00007B031F910F9108958091FD049091FE0416
:103A1000813A91050CF40AC38091D2078B3F98F04C
:103A20008B3F19F4809158050EC08C3F19F480919A
:103A30005A0509C08D3F19F480915C0504C08E3F82
:103A400021F480915E058093830380918303882312
:103A500019F41092830304C08F3F11F48093830301
:103A60008091D1078B3F98F08B3F19F480915805D6
:103A70000EC08C3F19F480915A0509C08D3F19F48E
:103A800080915C0504C08E3F21F480915E05809397
:103A9000820380918203882319F41092820305C067
:103AA000843618F084E6809382038091D3078B3F9D
:103AB00098F08B3F19F4809158050EC08C3F19F493
:103AC00080915A0509C08D3F19F480915C0504C0AE
:103AD0008E3F21F480915E0580938403809184035E
:103AE000882319F41092840305C0843618F084E604
:103AF000809384038091D5078B3F98F08B3F19F416
:103B0000809158050EC08C3F19F480915A0509C068
:103B10008D3F19F480915C0504C08E3F21F48091A3
:103B20005E058093850380918503882319F41092A4
:103B3000850304C08F3F11F4809385038091DC07D7
:103B40008B3F98F08B3F19F4809158050EC08C3F45
:103B500019F480915A0509C08D3F19F480915C05D4
:103B600004C08E3F21F480915E058093860380918E
:103B70008603882319F41092860304C08F3F11F442
:103B8000809386038091DD078B3F98F08B3F19F47B
:103B9000809158050EC08C3F19F480915A0509C0D8
:103BA0008D3F19F480915C0504C08E3F21F4809113
:103BB0005E0580938703809187038B3010F48AE041
:103BC00002C08F3F11F4809387038091DE078B3F03
:103BD00098F08B3F19F4809158050EC08C3F19F472
:103BE00080915A0509C08D3F19F480915C0504C08D
:103BF0008E3F21F480915E05809388038091880335
:103C0000882319F41092880304C08F3F11F4809325
:103C100088038091E3078B3F98F08B3F19F48091E4
:103C200058050EC08C3F19F480915A0509C08D3F8C
:103C300019F480915C0504C08E3F21F480915E05EB
:103C400080938A0380918A03882319F410928A034F
:103C500004C08F3F11F480938A038091E4078B3F67
:103C600098F08B3F19F4809158050EC08C3F19F4E1
:103C700080915A0509C08D3F19F480915C0504C0FC
:103C80008E3F21F480915E0580938B0380918B039E
:103C9000882319F410928B0304C08F3F11F4809392
:103CA0008B038091E5078B3F98F08B3F19F480914F
:103CB00058050EC08C3F19F480915A0509C08D3FFC
:103CC00019F480915C0504C08E3F21F480915E055B
:103CD00080938C0380918C03882319F410928C03B9
:103CE00004C08F3F11F480938C038091E6078B3FD3
:103CF00098F08B3F19F4809158050EC08C3F19F451
:103D000080915A0509C08D3F19F480915C0504C06B
:103D10008E3F21F480915E0580938D0380918D0309
:103D2000882319F410928D0304C08F3F11F48093FF
:103D30008D038091E7078B3F98F08B3F19F48091BA
:103D400058050EC08C3F19F480915A0509C08D3F6B
:103D500019F480915C0504C08E3F21F480915E05CA
:103D600080938E0380918E03882319F410928E0322
:103D700004C08F3F11F480938E038091F7078B3F2F
:103D800098F08B3F19F4809158050EC08C3F19F4C0
:103D900080915A0509C08D3F19F480915C0504C0DB
:103DA0008E3F21F480915E0580938F0380918F0375
:103DB000882319F410928F0304C08F3F11F480936D
:103DC0008F038091F8078B3F98F08B3F19F4809117
:103DD00058050EC08C3F19F480915A0509C08D3FDB
:103DE00019F480915C0504C08E3F21F480915E053A
:103DF0008093900380919003882319F4109290038C
:103E000004C08F3F11F4809390038091F9078B3F9A
:103E100098F08B3F19F4809158050EC08C3F19F42F
:103E200080915A0509C08D3F19F480915C0504C04A
:103E30008E3F21F480915E058093910380919103E0
:103E4000882319F41092910304C08F3F11F48093DA
:103E500091038091FA078B3F98F08B3F19F4809182
:103E600058050EC08C3F19F480915A0509C08D3F4A
:103E700019F480915C0504C08E3F21F480915E05A9
:103E80008093920380919203882319F410929203F5
:103E900004C08F3F11F4809392038091E8078B3F19
:103EA00098F08B3F19F4809158050EC08C3F19F49F
:103EB00080915A0509C08D3F19F480915C0504C0BA
:103EC0008E3F21F480915E0580939303809193034C
:103ED000882319F41092930304C08F3F11F4809348
:103EE00093038091ED078B3F98F08B3F19F48091FD
:103EF00058050EC08C3F19F480915A0509C08D3FBA
:103F000019F480915C0504C08E3F21F480915E0518
:103F10008093940380919403882319F4109294035E
:103F200004C08F3F11F4809394038091F0078B3F7E
:103F300098F08B3F19F4809158050EC08C3F19F40E
:103F400080915A0509C08D3F19F480915C0504C029
:103F50008E3F21F480915E058093950380919503B7
:103F6000882319F41092950304C08F3F11F48093B5
:103F700095038091F1078B3F98F08B3F19F4809166
:103F800058050EC08C3F19F480915A0509C08D3F29
:103F900019F480915C0504C08E3F21F480915E0588
:103FA0008093960380919603882319F410929603C8
:103FB00004C08F3F11F4809396038091F6078B3FE6
:103FC00098F08B3F19F4809158050EC08C3F19F47E
:103FD00080915A0509C08D3F19F480915C0504C099
:103FE0008E3F21F480915E05809397038091970323
:103FF000882319F41092970304C08F3F11F4809323
:10400000970360918A0370E080E090E00E942B3B70
:1040100027E137EB41ED58E30E94903E60937E0329
:1040200070937F0380938003909381030895809120
:104030005405882361F51092BF071092B6071092BD
:10404000A1071092AC071092AD071092C60780919D
:10405000BA04882331F08093AC078091AC07809339
:10406000B6078091BB04882331F08093A10780912B
:10407000A1078093BF078091BC04882311F080932F
:10408000C6078091BD04882311F08093AD0710927C
:10409000FA041092FB040E942315089510920F0554
:1040A00010920E05109211051092100580E090E01C
:1040B000A0E0B0E08093120590931305A09314053F
:1040C000B09315051092050510920405109207058E
:1040D000109206051092090510920805109295039A
:1040E000109296030E94931C84E690E00E949F0B1E
:1040F0000E94931C8091CF0780FF10C080910E0317
:1041000090910F03875B934038F480910E03909158
:104110000F038E5E924010F40E94AE0F8091D40483
:104120009091D50490930505809304058091D60461
:104130009091D70490930705809306058091D80449
:104140009091D90490930905809308058091060504
:104150009091070590930B0580930A0580910405C3
:104160009091050590930D0580930C0584E00E94C5
:1041700009388050944058F18091C0079091C10750
:1041800097FF03C0909581959F4F6CE070E00E946F
:10419000323F709311056093100580919B079091B9
:1041A0009C0797FF03C0909581959F4F6CE070E04E
:1041B0000E94323F70930F0560930E056091D20408
:1041C0007091D304882777FD8095982F17C084E0DD
:1041D0000E94093890930F0580930E0586E00E9497
:1041E0000938909311058093100588E00E940938E2
:1041F000AA2797FDA095BA2FBC01CD010E94D83DFA
:104200006093120570931305809314059093150520
:1042100010922A0510922B0510922C0510922D0554
:1042200010922E0510922F05109230051092310534
:104230001092320510923305109234051092350514
:1042400010923605109237051092380510923905F4
:1042500010923A0510923B0510923C0510923D05D4
:104260001092BE071092BD071092B3071092B207CA
:104270001092B5071092B40780910A0390910B0336
:10428000A0910C03B0910D039093510780935007B8
:104290001092E1041092E004109246051092470536
:1042A000109248051092490580916E0390916F031A
:1042B000909371038093700382E390E09093CE0417
:1042C0008093CD046091F20770E080E090E024ECF0
:1042D00039E040E050E00E94F33E6856754C8F4F45
:1042E0009F4F60937403709375038093760390934C
:1042F00077036091F30770E080E090E00E94F33E66
:104300006856754C8F4F9F4F609378037093790375
:1043100080937A0390937B0310927D0310927C0329
:10432000109271051092700510927305109272052B
:1043300060916E0370916F03882777FD8095982FA9
:104340002EE036E040E050E00E94F33E6093B70775
:104350007093B8078093B9079093BA071092BC077F
:104360001092BB0708951F93182F0EC0809154051B
:10437000882361F484E690E09093CE048093CD048A
:104380008AEF90E00E94BE0B115080F71F910895B4
:104390008091C707E82FF0E0EE0FFF1FE15AF84FBA
:1043A000808191818D5E9F4F14F0109298038081DF
:1043B00091818A5B9F4FDCF4809198038823B9F444
:1043C00081E08093980380914C058F5F80934C052A
:1043D00080914C05853028F480914C050E94B321D2
:1043E000089588EE93E09093CE048093CD040895D1
:1043F0002F923F924F925F926F927F928F929F92F5
:10440000AF92BF92CF92DF92EF92FF920F931F93E2
:10441000CF93DF93CDB7DEB7A2970FB6F894DEBF88
:104420000FBECDBF0E946417299A20916E0530916E
:104430006F058091D907482F50E0465F5F4F5A873C
:1044400049874217530714F43A8729878091FD045E
:104450009091FE04883791050CF071C080910301A2
:10446000882399F480910403909105038F5F9F4FF7
:1044700061F488E99AE39093CE048093CD0480E0C0
:104480009CE090930503809304038091AB05909189
:10449000AC05009731F001979093AC058093AB0584
:1044A00004C01092540510925505809100018A3085
:1044B00011F4289A01C028988091560590915705CB
:1044C000895E934008F401C48091E007A82FB0E012
:1044D000BA87A98781E080935505E091C7072E2F01
:1044E00030E0220F331FF901E358F84F1182108298
:1044F000A091C807B0E0AA0FBB1FFD01E358F84F19
:1045000011821082E091CA074E2F50E0440F551FD0
:10451000CA018358984FFC0111821082215A384FEA
:10452000F90111821082A15AB84F11961C921E9265
:10453000415A584FDA0111961C921E92CBC38091BA
:10454000FD049091FE048D3891050CF4C3C31092C4
:1045500055058091E10722E3829FC00111249093C9
:10456000AC058093AB05E985FA85B9976CF080912D
:10457000560590915705FFEF8F3F9F0729F0019651
:104580009093570580935605809156059091570555
:104590008F3F910509F0E8F41092BD051092BE0519
:1045A0001092BF051092C0051092B9051092BA057D
:1045B0001092BB051092BC0510926D0510926C050F
:1045C0008A3F910531F481E090E09093A3058093B8
:1045D000A20520915805309159058091CB07E82F0D
:1045E000F0E0EE0FFF1FE15AF84F80819181825970
:1045F0009F4F281739071CF42F5F3F4F0CC0808155
:10460000918182599F4F821793074CF421153105F0
:1046100031F02150304030935905209358052091B6
:104620005A0530915B058091CC07E82FF0E0EE0F42
:10463000FF1FE15AF84F8081918182599F4F2817BF
:1046400039071CF42F5F3F4F0CC080819181825944
:104650009F4F821793074CF42115310531F02150FB
:10466000304030935B0520935A0520915C053091D2
:104670005D058091CD07E82FF0E0EE0FFF1FE15AB6
:10468000F84F8081918182599F4F281739071CF478
:104690002F5F3F4F0CC08081918182599F4F8217BD
:1046A00093074CF42115310531F0215030403093FF
:1046B0005D0520935C0520915E0530915F0580913A
:1046C000CE07E82FF0E0EE0FFF1FE15AF84F808190
:1046D000918182599F4F281739071CF42F5F3F4F54
:1046E0000CC08081918182599F4F821793074CF4AF
:1046F0002115310531F02150304030935F05209372
:104700005E0520916005309161058091710790915F
:10471000720782599F4F281739071CF42F5F3F4FAC
:104720000EC0809171079091720782599F4F821736
:1047300093074CF42115310531F02150304030936E
:104740006105209360052091620530916305809199
:1047500073079091740782599F4F281739071CF4EB
:104760002F5F3F4F0EC0809173079091740782595D
:104770009F4F821793074CF42115310531F02150DA
:104780003040309363052093620520916405309199
:104790006505809175079091760782599F4F28177C
:1047A00039071CF42F5F3F4F0EC080917507909121
:1047B000760782599F4F821793074CF421153105D4
:1047C00031F02150304030936505209364052091ED
:1047D0006605309167058091770790917807825937
:1047E0009F4F281739071CF42F5F3F4F0EC0809151
:1047F00077079091780782599F4F821793074CF45F
:104800002115310531F02150304030936705209358
:104810006605809158059091590597FF05C0109243
:104820005905109258050AC08F3F910539F034F0B0
:104830008FEF90E0909359058093580580915A0529
:1048400090915B0597FF05C010925B0510925A0589
:104850000AC08F3F910539F034F08FEF90E09093CC
:104860005B0580935A0580915C0590915D0597FFEB
:1048700005C010925D0510925C050AC08F3F91053E
:1048800039F034F08FEF90E090935D0580935C05F4
:1048900080915E0590915F0597FF05C010925F05BE
:1048A00010925E050AC08F3F910539F034F08FEF0A
:1048B00090E090935F0580935E05809160059091F4
:1048C000610597FF05C010926105109260050AC04E
:1048D0008F3F910539F034F08FEF90E090936105B0
:1048E00080936005809162059091630597FF05C0F4
:1048F00010926305109262050AC08F3F910539F04E
:1049000034F08FEF90E0909363058093620580917F
:1049100064059091650597FF05C01092650510929A
:1049200064050AC08F3F910539F034F08FEF90E0B5
:104930009093650580936405809166059091670565
:1049400097FF05C010926705109266050AC08F3F59
:10495000910539F034F08FEF90E0909367058093E4
:104960006605E091C907F0E0EE0FFF1FE15AF84F2E
:1049700080819181813591050CF40EC1809154059F
:10498000882309F009C18091CA07E82FF0E0EE0FF3
:10499000FF1FE15AF84F808191818C3491050CF40E
:1049A000BFC08091AA058F5F8093AA05893C08F457
:1049B000F3C01092AA052998109257051092560537
:1049C0008091C707282F30E0D901AA0FBB1FA15A39
:1049D000B84F8D919C911197873491059CF48091EB
:1049E000C807E82FF0E0EE0FFF1FE15AF84F808173
:1049F000918197FF03C0909581959F4F87349105D2
:104A00000CF46BC08091C807682F70E0DB01AA0F1F
:104A1000BB1FA15AB84F8D919C9111978734910576
:104A20003CF0F901EE0FFF1FE15AF84F80819181B0
:104A30008D919C918734910564F0F901EE0FFF1F71
:104A4000E15AF84F808191818734910514F042E05A
:104A500001C041E0FB01EE0FFF1FE15AF84F8081DA
:104A60009181863491055CF4F901EE0FFF1FE15A44
:104A7000F84F80819181873491050CF043E0FB0170
:104A8000EE0FFF1FE15AF84F808191818A5B9F4FA3
:104A90005CF4F901EE0FFF1FE15AF84F808191811C
:104AA000873491050CF044E0660F771F615A784F08
:104AB000DB018D919C918A5B9F4F5CF4220F331F29
:104AC000215A384FF90180819181863491050CF487
:104AD00045E0842F0E9419381CC08091CF0783FFC6
:104AE00018C08081918197FF03C0909581959F4F59
:104AF00044977CF48D919C918A5B9F4F54F481E0A4
:104B000080934C0588EE93E09093CE048093CD047F
:104B100043C00E94FA390E9437380E944E2035C0A7
:104B200080819181855B9F4FACF58091AA058F5F55
:104B30008093AA05893C80F11092AA0529986FEF0D
:104B40007FEF84E00E9411381092570510925605AD
:104B50000E944E2060910E0570910F0584E00E9426
:104B60001138609110057091110586E00E9411388E
:104B700060911205709113058091140590911505AF
:104B80000E94AA3D88E00E9411380E94FA390E94D2
:104B9000B32102C01092AA05E091C907F0E0EE0F20
:104BA000FF1FE15AF84F808191818B5A9F4F0CF083
:104BB00091C08091CA07482F50E0FA01EE0FFF1F05
:104BC000E15AF84F80819181855B9F4F0CF064C062
:104BD0008091A9058F5F8093A905893C08F45EC088
:104BE0001092A90581E090E09093570580935605B7
:104BF00081E0809354051092B5051092B60510928D
:104C0000B7051092B80510923A0510923B05109224
:104C10003C0510923D0510922A0510922B0510922A
:104C20002C0510922D05109232051092330510922A
:104C30003405109235058091160590911705A091C5
:104C40001805B091190580932E0590932F05A09318
:104C50003005B093310580911E0590911F05A091FC
:104C60002005B09121058093360590933705A093D8
:104C70003805B09339051092BD051092BE0510920B
:104C8000BF051092C0051092B9051092BA05109296
:104C9000BB051092BC0502C01092A905440F551F18
:104CA000415A584FDA018D919C918C34910584F0D2
:104CB0008091A8058F5F8093A805893C58F01092D9
:104CC000A80510925705109256051092540502C07F
:104CD0001092A80580916B03815080936B038091A3
:104CE0006B038F3F29F080915505882309F477C322
:104CF0000E94041DE0916805F0916905FAA3E9A3FB
:104D00008091C707E82EFF24D701AA0FBB1FCD0152
:104D1000815A984FFC018081918198A38F8F809157
:104D2000D607682E7724A358B84F0D90BC91A02DBC
:104D3000BE8FAD8F8091D707A82EBB242091700520
:104D4000309171053C8F2B8F20906A0530906B0558
:104D50008091C807082F10E0C801880F991FDC0157
:104D6000A15AB84F0D90BC91A02DBA8FA98F83582E
:104D7000984FDC018D919C91988F8F8BE0917205FB
:104D8000F0917305FE8BED8BE091CA07AE2FB0E07A
:104D9000AA0FBB1FA15AB84F0D90BC91A02DBC8B80
:104DA000AB8BE091C907F0E0EE0FFF1FE15AF84F1F
:104DB000C080D18028E730E0C20ED31ED0926F05AC
:104DC000C0926E056091870370E080E090E00E94E1
:104DD0002B3B20E030E040E251E40E94D93C20E04F
:104DE00030E040E85CE30E94903E6F87788B898BCF
:104DF0009A8B6093C2077093C3078093C407909304
:104E0000C5076091880370E080E090E00E942B3B32
:104E100020E030EE4BE256E40E943D3D6093AE0749
:104E20007093AF078093B0079093B1072091BF04B0
:104E3000222331F08AE090E09093CE048093CD0459
:104E4000E22F22FF09C080919203482F50E0440FC7
:104E5000551F440F551F10C023FD03C040E050E014
:104E60000BC08091920390E0880F991F880F991FC3
:104E700044275527481B590B209178053091790517
:104E8000C901B3E0880F991FBA95E1F7821B930B14
:104E9000840F951F68E070E00E94323F2B017093F1
:104EA000790560937805E4FF09C080919203482F4B
:104EB00050E0440F551F440F551F10C0E5FD03C0BF
:104EC00040E050E00BC08091920390E0880F991F62
:104ED000880F991F44275527481B590B80917A0545
:104EE00090917B059C01E3E0220F331FEA95E1F7E7
:104EF000281B390BCA01820F931F68E070E00E94E3
:104F0000323F4B0170937B0560937A058091BE041C
:104F1000282F83FF03C082E390E004C082FF07C014
:104F20008EEC9FEF90937D0580937C0504C01092DA
:104F30007D0510927C0521FF09C080917C03909132
:104F40007D03019690937D0380937C0324FF09C029
:104F500080917C0390917D03019790937D038093D2
:104F60007C034F8D58A1469DC001479D900D569DD5
:104F7000900D112429A13AA1220F331F69A17AA112
:104F8000260F371FED8DFE8DEA9DD001EB9DB00DF4
:104F9000FA9DB00D11244B8D5C8DA41BB50BBAA3EB
:104FA000A9A3820F931F64E070E00E94323F89A1A1
:104FB0009AA1860F971F9AA389A3C20162E070E0AD
:104FC0000E94323FA9A1BAA1A60FB71FBAA3A9A3F5
:104FD000B0936905A0936805E98DFA8DE69DC0013F
:104FE000E79D900DF69D900D11249101220F331F26
:104FF000220D331D4F89588DB501469F5001479FA3
:10500000B00C569FB00C1124AD89BE89AA1ABB0AF8
:10501000820F931F64E070E00E94323FA60EB71E1D
:10502000C40162E070E00E94323FA60EB71EB0924B
:105030006B05A0926A0520917C0530917D05220FB9
:10504000331F220F331FEB89FC892E1B3F0B30933C
:105050006D0520936C058091750680FF56C0809188
:105060009203813808F451C080916E06992787FD1C
:105070009095AC01469DC001479D900D569D900DA9
:10508000112469A17AA1680F791F70936905609353
:10509000680580916F06992787FD9095DC01A69D94
:1050A000C001A79D900DB69D900D1124A80EB91EAC
:1050B000B0926B05A0926A0580917006992787FDD2
:1050C0009095280F391F30936D0520936C05209122
:1050D000D40730E080917206992787FD9095FC01F6
:1050E0002E9FC0012F9F900D3E9F900D11249093F5
:1050F0007D0380937C038091710690E08C159D0563
:1051000024F490936F0580936E0580916E059091C5
:105110006F0597FF04C010926F0510926E05809185
:10512000CF0782FF0CC080E090E0A0E0B0E0809369
:10513000AE079093AF07A093B007B093B10720E0FC
:1051400030E040E050E06F85788989899A890E9433
:10515000133E882364F480E090E0A0E0B0E0809308
:10516000C2079093C307A093C407B093C50720E07C
:1051700030E040E050E06091AE077091AF07809161
:10518000B0079091B1070E94133E882364F480E039
:1051900090E0A0E0B0E08093AE079093AF07A093BB
:1051A000B007B093B107E0916805F09169052091CF
:1051B000740530917505CF0164E070E00E94323FC4
:1051C00077FF03C0709561957F4F261737077CF4F2
:1051D000CF01F7FF03C0909581959F4F64E070E089
:1051E0000E94323F709375056093740506C021508C
:1051F00030403093750520937405E0916A05F09175
:105200006B052091760530917705CF0164E070E061
:105210000E94323F77FF03C0709561957F4F26173C
:1052200037077CF4CF01F7FF03C0909581959F4F1E
:1052300064E070E00E94323F7093770560937605DA
:1052400006C0215030403093770520937605F80151
:10525000EE0FFF1FE15AF84F208131818091EE0758
:10526000482F50E04217530744F48091FB0782FF18
:1052700004C081E08093880515C08091880588234B
:1052800089F0F801EE0FFF1FE15AF84F20813181BC
:105290008091EF07BA01681B71092617370714F4CC
:1052A00010928805F801EE0FFF1FE15AF84F808138
:1052B000918166277727641B750B8617970744F43F
:1052C0008091FB0783FF04C081E08093890515C0AE
:1052D00080918905882389F0000F111F015A184F0A
:1052E000D8012D913C918091EF0790E0841B950BA4
:1052F0008217930714F410928905F701EE0FFF1F30
:10530000E15AF84F808191814817590744F4809100
:10531000FB0780FF04C081E080938B0515C080915E
:105320008B05882389F0F701EE0FFF1FE15AF84F34
:10533000208131818091EF07FA01E81BF1092E17D6
:105340003F0714F410928B05F701EE0FFF1FE15A8F
:10535000F84F808191818617970744F48091FB076D
:1053600081FF04C081E080938A0517C080918A057F
:10537000882399F0EE0CFF1C2FE537E0E20EF31EB8
:10538000D7012D913C918091EF0790E0841B950B04
:105390008217930714F410928A0580918805882358
:1053A00021F480918905882321F081E0809387058D
:1053B00002C01092870580918B05882321F480918B
:1053C0008A05882351F081E0809386051092870535
:1053D000109288051092890502C01092860580916E
:1053E0008705882321F480918605882351F08091D8
:1053F000ED0790E0E985FA858E179F0714F49A87E8
:1054000089878091910390E09093F3048093F20454
:105410008091920390E09093F5048093F4040E94AD
:10542000BF1480915505882381F110926D0510926B
:105430006C05109269051092680510926B05109228
:105440006A0580E090E0A8ECBFE38093C2079093E8
:10545000C307A093C407B093C5078BE09CEBA2E3FE
:10546000BCE38093AE079093AF07A093B007B093CF
:10547000B10710928705109286051092750510925B
:105480007405109277051092760520919D07309152
:105490009E0740919F075091A0078091160590911B
:1054A0001705A0911805B0911905820F931FA41F2D
:1054B000B51F80939D0790939E07A0939F07B0937D
:1054C000A0072091A4073091A5074091A60750910D
:1054D000A70780911E0590911F05A0912005B0910E
:1054E0002105820F931FA41FB51F8093A4079093DB
:1054F000A507A093A607B093A7075090860555204F
:1055000029F480918705882309F44FC01092E304A1
:105510001092E20410923E0510923F051092400551
:1055200010924105109242051092430510924405D5
:105530001092450510929D0710929E0710929F07AA
:105540001092A0071092A4071092A5071092A60728
:105550001092A70780912A0590912B05A0912C0508
:10556000B0912D0580932E0590932F05A0933005C3
:10557000B09331058091320590913305A0913405A7
:10558000B09135058093360590933705A093380583
:10559000B093390510928505109284051092830509
:1055A00010928205552009F0F5C080918705882367
:1055B00009F0F0C0609116057091170580911805EB
:1055C00090911905A090DB07BB24CC24DD24E0904A
:1055D0009B07F0909C07A60195010E94673F00275A
:1055E000F7FC0095102F2E193F09400B510BCA01F3
:1055F000B90120E130E040E050E00E94673F39010E
:105600004A0160911E0570911F05809120059091BF
:105610002105E090C007F090C107A60195010E9406
:10562000673F0027F7FC0095102F2E193F09400B0C
:10563000510BCA01B90120E130E040E050E00E9486
:10564000673F79018A018091740590917505819772
:1056500034F480917605909177058197A4F0C40188
:10566000B30123E030E040E050E00E94673F3901A1
:105670004A01C801B70123E030E040E050E00E9459
:10568000673F79018A01E091CA07F0E0EE0FFF1F42
:10569000E15AF84F0190F081E02DF7FF03C0F0953B
:1056A000E195FF4F7A97A4F0C401B30123E030E005
:1056B00040E050E00E94673F39014A01C801B7014C
:1056C00023E030E040E050E00E94673F79018A012A
:1056D000F1E26F1671048104910434F070E2672ED8
:1056E000712C812C912C11C020EE62162FEF7206C6
:1056F0002FEF82062FEF920644F460EE662E6FEFD6
:10570000762E6FEF862E6FEF962E31E2E316F104C0
:105710000105110534F050E2E52EF12C012D112D7B
:1057200011C040EEE4164FEFF4064FEF04074FEFC1
:10573000140744F440EEE42E4FEFF42E4FEF042F05
:105740004FEF142F80912A0590912B05A0912C05E5
:10575000B0912D0586199709A809B90980932A05E2
:1057600090932B05A0932C05B0932D0580913205C5
:1057700090913305A0913405B09135058E199F099C
:10578000A00BB10B8093320590933305A0933405A1
:10579000B09335058091E2049091E3048F3F910529
:1057A00009F008F445C4552009F0DCC38091870551
:1057B000882309F0D7C380914D05882309F0D2C30F
:1057C00060919D0770919E0780919F079091A0071F
:1057D00020E031E040E050E00E94673F20939D07C9
:1057E00030939E0740939F075093A0076091A407B2
:1057F0007091A5078091A6079091A70720E031E05E
:1058000040E050E00E94673F2093A4073093A50733
:105810004093A6075093A707E090DB07FF2400E022
:1058200010E020913E0530913F0540914005509198
:105830004105C801B7010E94F33E20E031E040E09D
:1058400050E00E94673F20933E0530933F05409310
:105850004005509341052091420530914305409108
:10586000440550914505C801B7010E94F33E20E070
:1058700031E040E050E00E94673F209342053093C2
:105880004305409344055093450560919D077091F1
:105890009E0780919F079091A00720913E0530912F
:1058A0003F054091400550914105E090F407FF24E9
:1058B00000E010E0621B730B840B950BA8019701AD
:1058C0000E94673FCA01B90120E031E040E050E0AA
:1058D0000E94673F6901309385052093840560919C
:1058E000A4077091A5078091A6079091A707209122
:1058F0004205309143054091440550914505621B96
:10590000730B840B950BA80197010E94673FCA0196
:10591000B90120E031E040E050E00E94673F89019A
:1059200030938305209382058091740590917505CD
:105930008197BCF4809176059091770581978CF4DE
:10594000E091CA07F0E0EE0FFF1FE15AF84F019017
:10595000F081E02DF7FF03C0F095E195FF4F7A97B6
:1059600094F0C60162E070E00E94323F70938505BA
:1059700060938405C80162E070E00E94323F70933A
:10598000830560938205E0901A05F0901B05009155
:105990001C0510911D058091160590911705A09189
:1059A0001805B0911905E81AF90A0A0B1B0BE092C9
:1059B000B105F092B2050093B3051093B405809140
:1059C0002E0590912F05A0913005B09131058E19CB
:1059D0009F09A00BB10B80932E0590932F05A093E8
:1059E0003005B093310560902205709023058090BA
:1059F00024059090250580911E0590911F05A0918A
:105A00002005B0912105681A790A8A0A9B0A6092DA
:105A1000AD057092AE058092AF059092B005809171
:105A2000360590913705A0913805B0913905861952
:105A30009709A809B9098093360590933705A09373
:105A40003805B09339052091BB073091BC07213848
:105A500031054CF0809108059091090501969093CD
:105A600009058093080520583F4F4CF480910805A4
:105A7000909109050197909309058093080510926C
:105A8000BC071092BB0781E090E09093990580934A
:105A9000980510929E0510929F051092A0051092F5
:105AA000A10580919D0790919E07A0919F07B091BD
:105AB000A007209190053091910540919205509159
:105AC0009305281B390B4A0B5B0B57FF07C05095FA
:105AD0004095309521953F4F4F4F5F4F20523E44A8
:105AE000404050400CF0C1C071E0E71670E1F7068D
:105AF00070E0070770E017070CF452C0809197051B
:105B0000882309F449C0D801C7012CE0B595A795B1
:105B1000979587952A95D1F701969093990580934B
:105B20009805D801C701F3E0B595A7959795879596
:105B3000FA95D1F780939E0590939F05A093A005B9
:105B4000B093A10589589341A040B04064F088E823
:105B500093E1A0E0B0E080939E0590939F05A09311
:105B6000A005B093A10560919E0570919F0580915D
:105B7000A0059091A10520E031E040E050E00E94B6
:105B8000673F8091840590918505820F931F9093C4
:105B900085058093840566C081E08093970562C087
:105BA00010929705F0E0EF16F0EFFF06FFEF0F07FA
:105BB000FFEF1F070CF056C080919605882309F46B
:105BC0004DC088279927DC018E199F09A00BB10BC6
:105BD000ECE0B595A79597958795EA95D1F701964D
:105BE0009093990580939805C801B70128E030E0AB
:105BF00040E050E00E94673F20939E0530939F0550
:105C00004093A0055093A10528573C4E4F4F5F4F3E
:105C100064F488E79CEEAFEFBFEF80939E0590930E
:105C20009F05A093A005B093A10560919E0570917A
:105C30009F058091A0059091A10520E031E040E012
:105C400050E00E94673F8091840590918505820F06
:105C5000931F909385058093840511C081E0809304
:105C600096050DC0109296050AC0109299051092E3
:105C7000980584EF91E09093730380937203809171
:105C8000F507C82EDD248091980590919905C816D6
:105C9000D90624F4D0929905C092980571E0E716D0
:105CA00074E0F70670E0070770E0170774F0809162
:105CB0000405909105052091980530919905820F72
:105CC000931F909305058093040580E0E8168CEF00
:105CD000F8068FEF08078FEF180774F4809104051A
:105CE000909105052091980530919905821B930BA1
:105CF000909305058093040581E090E090939905C9
:105D00008093980510929A0510929B0510929C051D
:105D100010929D058091A4079091A507A091A607D8
:105D2000B091A70720918C0530918D0540918E058B
:105D300050918F05281B390B4A0B5B0B57FF07C08F
:105D400050954095309521953F4F4F4F5F4F2052D2
:105D50003E44404050400CF0C1C0A1E06A16A0E1B2
:105D60007A06A0E08A06A0E09A060CF452C0809160
:105D70009505882309F449C0D401C3017CE0B59599
:105D8000A795979587957A95D1F701969093990560
:105D900080939805D401C30163E0B595A7959795C5
:105DA00087956A95D1F780939A0590939B05A09368
:105DB0009C05B0939D0589589341A040B04064F084
:105DC00088E893E1A0E0B0E080939A0590939B056A
:105DD000A0939C05B0939D0560919A0570919B05D9
:105DE00080919C0590919D0520E031E040E050E0DD
:105DF0000E94673F8091820590918305820F931FD7
:105E0000909383058093820566C081E08093950519
:105E100062C010929505F0E06F16F0EF7F06FFEF7D
:105E20008F06FFEF9F060CF056C0809194058823E3
:105E300009F44DC088279927DC0186199709A8091C
:105E4000B9095CE0B595A795979587955A95D1F7CF
:105E500001969093990580939805C401B30128E0B9
:105E600030E040E050E00E94673F20939A05309375
:105E70009B0540939C0550939D0528573C4E4F4FE2
:105E80005F4F64F488E79CEEAFEFBFEF80939A0515
:105E900090939B05A0939C05B0939D0560919A05F6
:105EA00070919B0580919C0590919D0520E031E0CB
:105EB00040E050E00E94673F809182059091830509
:105EC000820F931F909383058093820511C081E018
:105ED000809394050DC0109294050AC01092990504
:105EE0001092980584EF91E090937303809372036E
:105EF0008091980590919905C816D90624F4D092FE
:105F00009905C092980571E0671674E0770670E015
:105F1000870670E0970674F080910605909107055A
:105F20002091980530919905820F931F9093070552
:105F30008093060580E068168CEF78068FEF880660
:105F40008FEF9806CCF4809106059091070520917B
:105F5000980530919905821B930B909307058093C8
:105F600006050AC0109283051092820510928505DD
:105F70001092840510924D0520E030E040E050E0A2
:105F80006091AE077091AF078091B0079091B10713
:105F90000E94133E882341F41092830510928205DB
:105FA000109285051092840580919D0790919E071F
:105FB000A0919F07B091A0078093900590939105C1
:105FC000A0939205B09393058091A4079091A507A3
:105FD000A091A607B091A70780938C0590938D059B
:105FE000A0938E05B0938F0510923E0510923F0549
:105FF00010924005109241051092420510924305FF
:10600000109244051092450510929D0710929E072C
:1060100010929F071092A0071092A4071092A50754
:106020001092A6071092A7071092E3041092E204C0
:10603000C0906C05D0906D058601D7FE04C0002786
:1060400011270C191D0900311105C4F08091CF07EB
:1060500084FD14C081E090E09093A3058093A20595
:106060008091B7079091B807909371038093700364
:106070008AEF90E09093730380937203E090D807C7
:10608000B601882777FD8095982F2E2D30E040E0CF
:1060900050E00E94F33E9801442737FD4095542F6D
:1060A0000E94F33E20E032E040E050E00E94673F73
:1060B00089019A01FF24EC9CC001ED9C900DFC9C91
:1060C000900D112464E070E00E94323F600F711F58
:1060D000882777FD8095982F6093B5057093B60556
:1060E0008093B7059093B80520913A0530913B0510
:1060F00040913C0550913D05261B370B480B590B31
:1061000020933A0530933B0540933C0550933D0561
:1061100080913A0590913B05A0913C05B0913D05D9
:106120008155934CA040B04064F080E593ECA0E032
:10613000B0E080933A0590933B05A0933C05B09363
:106140003D0580913A0590913B05A0913C05B091A9
:106150003D05805B9C43AF4FBF4F64F480EB9CE3F5
:10616000AFEFBFEF80933A0590933B05A0933C05BA
:10617000B0933D058091CF0783FF5AC180914C05B4
:10618000882339F080915405882319F40E94C8218E
:106190004FC1609116057091170580911805909177
:1061A000190520E032E040E050E00E94673F89019D
:1061B00037FF03C0109501951F4F60911E05709128
:1061C0001F05809120059091210520E032E040E0FC
:1061D00050E00E94673F690137FF04C0D094C1942A
:1061E000D108D394C016D1060CF4680129E1C21677
:1061F000D10444F58091A2059091A305892B11F15A
:106200008091720390917303892BE1F488EC90E004
:106210009093CE048093CD046091B7077091B80736
:106220008091B9079091BA072EE036E040E050E047
:106230000E94673F30937103209370031092A3056F
:106240001092A20580916E0390916F0397FF03C097
:1062500020E030E029C0E0906E03F0906F034CE145
:1062600052E0E40EF51E0027F7FC0095102F609118
:10627000B7077091B8078091B9079091BA072EE0DF
:1062800036E040E050E00E94673FE21AF30A040B58
:10629000150BC801B70128E631E040E050E00E944C
:1062A000673F9B01245B3040C60168E070E00E94BC
:1062B000323F6F5F7F4FC90143E0880F991F4A95B6
:1062C000E1F70E94323F3B01882477FC8094982CB0
:1062D0008091B7079091B807A091B907B091BA071C
:1062E000680E791E8A1E9B1E6092B7077092B807CF
:1062F0008092B9079092BA0780918603A82EBB249A
:10630000CA9CC001CB9C900DDA9C900D112460E4D6
:1063100070E00E94323F2501461A570A14141504F2
:106320000CF080C08091720390917303009711F07C
:1063300001977AC08091BB079091BC07820F931F91
:106340009093BC078093BB07809176059091770569
:106350002091740530917505820F931F68E070E0FD
:106360000E94323F6B0160E470E0C60ED71E809140
:10637000700390917103AA2797FDA095BA2F0CE1A5
:10638000E02E02E0F02E012D112DE81AF90A0A0B79
:106390001B0BC401B3012EE036E040E050E00E9448
:1063A000673FE20EF31E041F151FC801B70128E660
:1063B00031E040E050E00E94673F645B7040649DC4
:1063C000C001659D900D749D900D1124B6010E9431
:1063D000323FC501880F991F8A0D9B1D86179707AD
:1063E00034F0909581959F4F681779070CF4BC01A4
:1063F00020913A0530913B0540913C0550913D0577
:10640000CB01AA2797FDA095BA2F820F931FA41F37
:10641000B51F80933A0590933B05A0933C05B0933C
:106420003D0506C08AEF90E090937303809372035A
:106430008091A40581508093A4058F3F09F0B4C0DA
:1064400088E18093A40560911605709117058091ED
:10645000180590911905E090DB07FF2400E010E09B
:10646000A80197010E94673F309379062093780630
:1064700060911E0570911F05809120059091210566
:10648000A80197010E94673F30937B0620937A060C
:1064900080919B0790919C0790937D0680937C064A
:1064A0008091C0079091C10790937F0680937E06EC
:1064B0008091B4079091B5079093810680938006F0
:1064C00080917E0590917F0590938306809382064C
:1064D0006091460570914705809148059091490566
:1064E00020E032E040E050E00E94673F30938506B4
:1064F000209384068091FD049091FE049093890678
:1065000080938806809108039091090390938B06ED
:1065100080938A068091B60790E090938D068093D1
:106520008C068091AC0790E090938F0680938E0646
:106530008091BF0790E090939106809390068091A0
:10654000A10790E090939306809392068091C607EE
:1065500090E090939506809394068091AD0790E02B
:1065600090939706809396068091AA079091AB0727
:1065700090939906809398068091D0049091D104CD
:106580009093A1068093A00680917005909171056B
:106590009093B5068093B40680917205909173052F
:1065A0009093B7068093B606809186058823A9F05C
:1065B0006091BD077091BE07882777FD8095982F61
:1065C0000E94D83D2091C2073091C3074091C40773
:1065D0005091C5070E94903E32C06091160570919F
:1065E00017058091180590911905E090BD07F0906E
:1065F000BE070E94D83D2091AE073091AF07409171
:10660000B0075091B1070E94903E5B016C010027DA
:10661000F7FC0095102FC801B7010E94D83D2091CA
:10662000C2073091C3074091C4075091C5070E942B
:10663000903E9B01AC01C601B5010E94D93C0E946D
:10664000A53D7093BE076093BD07809187058823A1
:10665000A9F06091B2077091B307882777FD809504
:10666000982F0E94D83D2091C2073091C3074091D6
:10667000C4075091C5070E94903E32C060911E052C
:1066800070911F058091200590912105E090B2073F
:10669000F090B3070E94D83D2091AE073091AF072C
:1066A0004091B0075091B1070E94903E5B016C0190
:1066B0000027F7FC0095102FC801B7010E94D83DB4
:1066C0002091C2073091C3074091C4075091C5077C
:1066D0000E94903E9B01AC01C601B5010E94D93CCD
:1066E0000E94A53D7093B3076093B2076091B40711
:1066F0007091B507A0902605B0902705C090280599
:10670000D09029058091AE079091AF07A091B00776
:10671000B091B10789839A83AB83BC83882777FDC7
:106720008095982F0E94D83D7B018C016091C20713
:106730007091C3078091C4079091C5079B01AC017C
:106740000E94D93C9B01AC01C801B7010E94903E58
:106750007B018C01C601B5010E94D83D29813A8197
:106760004B815C810E94903E20E030E040E05FE39E
:106770000E94903E9B01AC01C801B7010E94D93C28
:106780000E94A53D7093B5076093B4078091BD0743
:106790009091BE079093A3068093A2068091B207C2
:1067A0009091B3079093A5068093A4068091BD07AE
:1067B0009091BE078150904434F080E090E4909333
:1067C000BE078093BD078091BD079091BE078050A2
:1067D000904C34F480E090EC9093BE078093BD071A
:1067E0008091B2079091B3078150904434F080E0DB
:1067F00090E49093B3078093B2078091B207909191
:10680000B3078050904C34F480E090EC9093B30741
:106810008093B2078091B4079091B507815090445E
:1068200034F080E090E49093B5078093B4078091B2
:10683000B4079091B5078050904C34F480E090EC10
:106840009093B5078093B407A984BA84AA0CBB1CA3
:10685000AA0CBB1C8091CF07282F80FFC7C0809156
:106860005505882309F0C2C08091830321FF0EC023
:10687000823310F580917E0590917F054497909327
:106880008105809380051092A70519C020917C0393
:1068900030917D03280F311D8091D40790E0AC0129
:1068A000249FC001259F900D349F900D1124449783
:1068B000909381058093800581E08093A7052091C6
:1068C0007E0530917F0540918005509181054217EA
:1068D00053070CF08BC08091A705882309F486C06C
:1068E0008091840390E0241B350BBC01629FC001A2
:1068F000639F900D729F900D112464E070E00E94E0
:10690000323F4B01C090E004D090E1046091460515
:10691000709147058091480590914905E090850365
:10692000FF2400E010E020E830E040E050E00E946A
:10693000673FC801B7010E94F33E20E230E040E02B
:1069400050E00E94673F7EEF283E370714F428EEA0
:106950003EEF8091A5059091A605FC01A4E0EE0F05
:10696000FF1FAA95E1F7E81BF90BC60162E070E092
:106970000E94323FE61BF70B81E02931380714F003
:1069800028E131E0E21BF30BC501881999098E0F4C
:106990009F1F60E170E00E94323F7093A6056093F4
:1069A000A5058091D00790E0880F991F880F991F47
:1069B0006817790764F4A816B9062CF09093A60519
:1069C0008093A50504C0B092A605A092A50580916C
:1069D000A5059091A605A816B90624F4B092A605BF
:1069E000A092A505A090A505B090A6058091DA0714
:1069F000882E99248401000F111F000F111FC80158
:106A000080559040BAA2A9A28A159B0514F49AA3B6
:106A100089A3A9A1BAA1B0938706A0938606209165
:106A2000B4073091B5078091B5059091B605A09156
:106A3000B705B091B80542E0880F991FAA1FBB1F88
:106A40004A95D1F7281B390BE9A1FAA1E13AF105E2
:106A5000ACF0F595E7952E173F070CF4F90189A1E5
:106A60009AA162E070E00E94323F709561957F4F7D
:106A7000CF01E617F7076CF4CB010BC0C901205B0F
:106A80003F4F14F480EB9FEF8135910514F080E5C2
:106A900090E0980149A15AA1241B350B281739070A
:106AA0000CF4C90129A13AA1201B310B2C0182173A
:106AB00093070CF429018091BD079091BE07609067
:106AC000680570906905861997099093A9078093C6
:106AD000A80720E030E040E050E069817A818B81B6
:106AE0009C810E94133E8823F1F1E0901605F090FE
:106AF000170500911805109119056091BD05709159
:106B0000BE058091BF059091C0050E94D83D5B01F4
:106B10006C01C801B7010E94D83D29813A814B819F
:106B20005C810E94903E7B018C01B301882777FD38
:106B30008095982F0E94D83D9B01AC01C801B701F8
:106B40000E94D83C9B01AC01C601B5010E94D93C12
:106B50000E94A53D6093BD057093BE058093BF055F
:106B60009093C0051CC02091A8073091A907442725
:106B700037FD4095542F8091BD059091BE05A091A1
:106B8000BF05B091C005820F931FA41FB51F80934E
:106B9000BD059093BE05A093BF05B093C00580913D
:106BA000BD059091BE05A091BF05B091C005815073
:106BB0009A4FA040B04064F080E09AEFA0E0B0E0CF
:106BC0008093BD059093BE05A093BF05B093C0050B
:106BD0008091BD059091BE05A091BF05B091C00503
:106BE00080509640AF4FBF4F64F480E096E0AFEF27
:106BF000BFEF8093BD059093BE05A093BF05B093F2
:106C0000C0056091A8077091A90780917E039091BB
:106C10007F03A0918003B09181038B879C87AD8710
:106C2000BE87882777FD8095982F0E94D83D7B01ED
:106C30008C016091BD057091BE058091BF0590915A
:106C4000C0050E94D83D9B01AC016B857C858D857C
:106C50009E850E94903E9B01AC01C801B7010E9435
:106C6000D93C0E94A53D7B018C016B01C20157FEFE
:106C700004C0882799278419950962E070E00E9472
:106C8000323FA9A1BAA16A0F7B1F882777FD8095A3
:106C9000982F2091970330E040E050E00E94F33EAF
:106CA00020E430E040E050E00E94673F3E832D83C7
:106CB000C216D3060CF497012D803E8030942194A7
:106CC0003108339438872F832215330514F438861E
:106CD0002F828091B2079091B30760906A057090FF
:106CE0006B05861997099093A3078093A20720E06C
:106CF00030E040E050E069817A818B819C810E9484
:106D0000133E8823F1F1E0901E05F0901F050091DD
:106D10002005109121056091B9057091BA05809107
:106D2000BB059091BC050E94D83D5B016C01C80178
:106D3000B7010E94D83D29813A814B815C810E9434
:106D4000903E7B018C01B301882777FD8095982FB9
:106D50000E94D83D9B01AC01C801B7010E94D83CFC
:106D60009B01AC01C601B5010E94D93C0E94A53D22
:106D70006093B9057093BA058093BB059093BC05E9
:106D80001CC02091A2073091A307442737FD4095EE
:106D9000542F8091B9059091BA05A091BB05B0918F
:106DA000BC05820F931FA41FB51F8093B905909354
:106DB000BA05A093BB05B093BC058091B90590912D
:106DC000BA05A091BB05B091BC0581509A4FA04077
:106DD000B04064F080E09AEFA0E0B0E08093B905A5
:106DE0009093BA05A093BB05B093BC058091B905FB
:106DF0009091BA05A091BB05B091BC05805096401A
:106E0000AF4FBF4F64F480E096E0AFEFBFEF8093E9
:106E1000B9059093BA05A093BB05B093BC056091EA
:106E2000A2077091A307882777FD8095982F0E946D
:106E3000D83D7B018C016091B9057091BA058091B4
:106E4000BB059091BC050E94D83D9B01AC016B85B0
:106E50007C858D859E850E94903E9B01AC01C8017A
:106E6000B7010E94D93C0E94A53D2D813E81621749
:106E700073070CF49B018101221633060CF489017F
:106E80002F81388549A15AA1240F351FC80162E01E
:106E900070E00E94323F7B01C901860F971F841961
:106EA000950964E070E00E94323F8616970614F45C
:106EB000B40107C08091D90790E0681779070CF4F6
:106EC000BC016093B607240D351DC9018E199F09B9
:106ED00064E070E00E94323F8616970614F4B40115
:106EE00007C08091D90790E0681779070CF4BC01BE
:106EF0006093AC0729A13AA16F817885261B370BD7
:106F0000C701820F931F8419950964E070E00E9405
:106F1000323F8616970614F4B40107C08091D90752
:106F200090E0681779070CF4BC016093BF07240D4B
:106F3000351DC9018E199F0964E070E00E94323F3F
:106F40008616970614F4B40107C08091D90790E023
:106F5000681779070CF4BC016093A10789A19AA175
:106F6000840D951D800F911F64E070E00E94323FF8
:106F70008616970614F4B40107C08091D90790E0F3
:106F8000681779070CF4BC016093C60789A19AA120
:106F9000801B910B9AA389A38419950964E070E082
:106FA0000E94323F8616970644F08091D90790E000
:106FB0004B01681779070CF44C018092AD07A2963B
:106FC0000FB6F894DEBF0FBECDBFDF91CF911F91FA
:106FD0000F91FF90EF90DF90CF90BF90AF909F9078
:106FE0008F907F906F905F904F903F902F9008957B
:106FF000A0E0B0E0A80FB11D0E94B93F802D90E045
:107000000895A0E0B0E0A80FB11D062E0E94CB3F6E
:107010000895A0E0B0E0A80FB11D0E94C63FCF01C7
:107020000895A0E0B0E0A80FB11D0B010E94D73F6A
:107030000895863008F085E0A2E0B0E0082E0E94B6
:10704000CB3F0895982F863008F095E086E4989F0E
:10705000D0011124AC59BF4FE7ECF7E0182E0E9485
:10706000DC3FA2E0B0E0092E0E94CB3F0895982FAC
:10707000863008F095E086E4989FD0011124AC5941
:10708000BF4FE7ECF7E0182E0E94C13F089581E062
:107090008093C70782E08093C80743E04093C90705
:1070A00064E06093CA0755E05093CB0736E0309315
:1070B000CC0787E08093CD0728E02093CE0788EEA9
:1070C0008093CF079EE19093D0078BEF8093D207F8
:1070D0008AE08093D3079093D1079093D50740938C
:1070E000D4072093D60740E14093D7073093D807C1
:1070F0002093D90786EE8093DA079093DB0780E828
:107100008093DC0734E63093DD0788E78093DE0761
:107110008EE58093DF0783E28093E00784E180932C
:10712000E1071092E2074093E3078DEF8093E407B5
:107130003093E5079AE59093E6079093E7079093DD
:10714000F7079093F8071092F9071092FA07309317
:10715000E80788E28093E9071092FC0722E3209376
:10716000EA0786E98093EB075093EC072093ED073D
:107170009093EE072093EF071092FB079093F00790
:107180005093F1073093F2073093F30780E2809336
:10719000F4076093F5072093F607A1E0B8E0E9E96A
:1071A000F3E089E001900D928150E1F7089581E0CC
:1071B0008093C70782E08093C80743E04093C907E4
:1071C00064E06093CA0755E05093CB0736E03093F4
:1071D000CC0787E08093CD0728E02093CE0788E690
:1071E0008093CF079EE19093D0078BEF8093D207D7
:1071F0008AE08093D3079093D1079093D50740936B
:10720000D4078CE08093D60780E18093D707309332
:10721000D8072093D90786EE8093DA079093DB078F
:1072200080E88093DC0780E58093DD0788E7809322
:10723000DE078EE58093DF0783E28093E00790937B
:10724000E1071092E20740E24093E3078DEF80935D
:10725000E40734E63093E5072AE52093E607209318
:10726000E7072093F7072093F8071092F907109289
:10727000FA073093E80788E28093E9071092FC0749
:1072800092E39093EA0786E98093EB075093EC072B
:107290009093ED072093EE079093EF071092FB0772
:1072A0002093F0075093F1073093F2073093F307E0
:1072B0004093F4076093F5078BE48093F607A1E011
:1072C000B8E0E3EAF3E087E001900D928150E1F746
:1072D000089581E08093C70782E08093C80783E028
:1072E0008093C90754E05093CA0735E03093CB0729
:1072F00086E08093CC0787E08093CD0728E0209339
:10730000CE0788E68093CF079EE19093D0078BEF5E
:107310008093D2078AE08093D3079093D10790930C
:10732000D5075093D4078FE08093D6079093D70763
:107330008CE08093D8072093D90786EE8093DA07F4
:107340009093DB0780E88093DC0780E58093DD077E
:1073500046E94093DE078EE58093DF0783E2809362
:10736000E0079093E1071092E20780E28093E30741
:107370008DEF8093E40724E62093E5079AE5909348
:10738000E6079093E7079093F7079093F80710921A
:10739000F9071092FA072093E80788E28093E9073B
:1073A0001092FC0782E38093EA074093EB07309347
:1073B000EC078093ED079093EE078093EF07109210
:1073C000FB079093F0073093F1072093F207209387
:1073D000F30780E18093F4075093F5072093F607B5
:1073E000A1E0B8E0EBEAF3E086E001900D92815075
:1073F000E1F7089522E030E0D9010E94B93F802DE5
:10740000863028F082E0D901082E0E94CB3F90E020
:1074100008950F931F93CF93DF93A1E0B0E00E94F4
:10742000B93F802D863469F18CE594E09F938F936A
:107430001F920E944D080E946939C0E0D0E00F9071
:107440000F900F900C2FC23039F0C33019F40E9406
:10745000473804C0C43010F00E94D738802F0E94F3
:1074600022382196C630D10569F7A2E0B0E083E06A
:10747000082E0E94CB3FA1E0B0E086E4082E0E94D7
:10748000CB3F02E010E0D8010E94B93F802D0E945E
:107490003738D8010E94B93F802D90E09F938F9399
:1074A00083E494E09F938F931F920E944D080F9066
:1074B0000F900F900F900F90DF91CF911F910F9130
:1074C0000895CF93DF93DC01EC01EA81FB812191E8
:1074D0008E81815019F48981E81BF109ED01FB834C
:1074E000EA838E839FB7F8948C9181508C939FBFD1
:1074F000822F90E0DF91CF910895FC011082758377
:107500006483738362834183478346830895CF9363
:10751000DF93DC019C91ED018981981718F080E0E0
:1075200090E016C0ED01EC81FD8161938F81815067
:1075300019F48981E81BF109ED018F83FD83EC8348
:107540009FB7F8948C918F5F8C939FBF81E090E000
:10755000DF91CF910895FC0180818823E9F3CF0169
:107560000E94613A90E00895FC018081882319F41B
:107570008FEF9FEF0895CF010E94613A90E0089548
:107580009FB7F8948091C9008F778093C90080914C
:10759000C9008F7B8093C9008091C9008F7D809343
:1075A000C9005A9A52985B9A539A1092CD008AE277
:1075B0008093CC008091C80082608093C80088E1ED
:1075C0008093C9008091CA008F778093CA00809110
:1075D000CA008F7B8093CA008091CA008F7D809300
:1075E000CA008091CA008F7E8093CA008091CA0031
:1075F000877F8093CA008091C9008B7F8093C900E8
:107600008091CA0084608093CA008091CA00826021
:107610008093CA0002C08091CE008091C80087FD8F
:10762000FACF8091C90080688093C9008091C90019
:1076300080648093C9009FBF08951F920F920FB678
:107640000F9211248F938091CE008F910F900FBED7
:107650000F901F901895A8E0B0E0E1E3FBE30C94D5
:107660008C3F7B018C01611571058105910519F431
:1076700082E089835AC083E089838EE1C82ED12CB1
:10768000DC82CB82ED82FE820F831887C801B701AE
:107690000E949E3BBC016150704077FF33C0EE27D3
:1076A000FF27E61BF70B20E030E040E050E081E0F0
:1076B00090E0A0E0B0E00E2E04C0880F991FAA1F32
:1076C000BB1F0A94D2F70197A109B1098E219F210E
:1076D000A023B1230097A105B10521F021E030E0FE
:1076E00040E050E004C016950795F794E794EA95BA
:1076F000D2F72E293F29402B512B2D833E834F83D8
:1077000058870FC06115710581F0062E04C0EE0C7C
:10771000FF1C001F111F0A94D2F7ED82FE820F8317
:107720001887C61AD70ADC82CB821A82CE0101964C
:107730000E94EB3BE8E028960C94A83FEF92FF9262
:107740000F931F939B01AC01203080E0380781E04C
:10775000480780E0580780F42F3F31054105510567
:1077600009F020F4EE24FF24870119C068E0E62E1A
:10777000F12C012D112D13C0203080E0380780E05E
:10778000480781E0580730F490E1E92EF12C012DF3
:10779000112D05C088E1E82EF12C012D112D80E27C
:1077A00090E0A0E0B0E08E199F09A00BB10B04C0DF
:1077B0005695479537952795EA94D2F7F901EE54F7
:1077C000FC4F2081821B9109A109B1091F910F91E2
:1077D000FF90EF9008959F92AF92BF92CF92DF9269
:1077E000EF92FF920F931F93EE24FF248701FC0179
:1077F000248135814681578191808081823010F4C7
:107800004061A2C0843009F49BC0823029F420E09A
:1078100030E040E050E005C021153105410551053B
:1078200019F4E0E0F0E092C0828193816FEF82383A
:1078300096070CF05AC062E87FEF681B790B6A313B
:1078400071052CF020E030E040E050E02AC0AA248E
:10785000BB24650181E090E0A0E0B0E0062E04C00A
:10786000880F991FAA1FBB1F0A94D2F70197A1097D
:10787000B10982239323A423B5230097A105B10561
:1078800029F071E0A72EB12CC12CD12C04C0569543
:107890004795379527956A95D2F72A293B294C2990
:1078A0005D29DA01C9018F779070A070B0708034C3
:1078B0009105A105B10539F427FF09C0205C3F4FB0
:1078C0004F4F5F4F04C0215C3F4F4F4F5F4F80E0F1
:1078D00090E0203060E0360760E0460760E456073D
:1078E00010F081E090E0FC0123C08038910544F560
:1078F000FC01E158FF4FDA01C9018F779070A07049
:10790000B07080349105A105B10539F427FF09C095
:10791000205C3F4F4F4F5F4F04C0215C3F4F4F4FA4
:107920005F4F57FF05C05695479537952795319678
:1079300087E056954795379527958A95D1F706C0E4
:1079400020E030E040E050E0EFEFF0E0E22EF32EF8
:10795000942F9F77802F8078892B9E2F979599273A
:1079600097958F77082F092B9E2F9695812F8078DA
:10797000892B9794992497948F77182F1929C801E8
:10798000B7011F910F91FF90EF90DF90CF90BF90C4
:10799000AF909F900895FC014150504030F001900D
:1079A0000616D1F73197CF010895882799270895B2
:1079B0005058BB27AA270ED079C16AD130F06FD1B9
:1079C00020F031F49F3F11F41EF45FC10EF4E095F6
:1079D000E7FB55C1E92F7BD180F3BA176207730724
:1079E0008407950718F071F49EF593C10EF4E095A5
:1079F0000B2EBA2FA02D0B01B90190010C01CA0169
:107A0000A0011124FF27591B99F0593F50F4503E13
:107A100068F11A16F040A22F232F342F4427585F05
:107A2000F3CF469537952795A795F0405395C9F71D
:107A30007EF41F16BA0B620B730B840BBAF09150D5
:107A4000A1F0FF0FBB1F661F771F881FC2F70EC074
:107A5000BA0F621F731F841F48F487957795679547
:107A6000B795F7959E3F08F0B3CF9395880F08F030
:107A70009927EE0F9795879508950CD017C10FD1D0
:107A800040F006D130F021F45F3F19F0F8C05111F9
:107A900041C1FBC01CD198F39923C9F35523B1F31D
:107AA000951B550BBB27AA2762177307840738F06D
:107AB0009F5F5F4F220F331F441FAA1FA9F333D0CC
:107AC0000E2E3AF0E0E830D091505040E695001C80
:107AD000CAF729D0FE2F27D0660F771F881FBB1F3C
:107AE000261737074807AB07B0E809F0BB0B802D16
:107AF000BF01FF2793585F4F2AF09E3F510568F062
:107B0000BEC008C15F3FECF3983EDCF386957795E5
:107B10006795B795F7959F5FC9F7880F911D969563
:107B2000879597F90895E1E0660F771F881FBB1FBF
:107B3000621773078407BA0720F0621B730B840B6C
:107B4000BA0BEE1F88F7E095089504D06894B11140
:107B5000E1C00895C4D088F09F5790F0B92F9927BD
:107B6000B751A0F0D1F0660F771F881F991F1AF048
:107B7000BA95C9F712C0B13081F0CBD0B1E0089509
:107B8000C8C0672F782F8827B85F39F0B93FCCF38A
:107B9000869577956795B395D9F73EF4909580953E
:107BA000709561957F4F8F4F9F4F0895E89409C05E
:107BB00097FB3EF490958095709561957F4F8F4F20
:107BC0009F4F9923A9F0F92F96E9BB279395F69536
:107BD000879577956795B795F111F8CFFAF4BB0FB4
:107BE00011F460FF1BC06F5F7F4F8F4F9F4F16C018
:107BF000882311F096E911C0772321F09EE8872FA2
:107C0000762F05C0662371F096E8862F70E060E05D
:107C10002AF09A95660F771F881FDAF7880F9695D6
:107C2000879597F9089507D008F481E0089503D067
:107C300008F48FEF0895990F0008550FAA0BE0E89C
:107C4000FEEF16161706E807F907C0F0121613061E
:107C5000E407F50798F0621B730B840B950B39F45E
:107C60000A2661F0232B242B252B21F408950A26C4
:107C700009F4A140A6958FEF811D811D089597F904
:107C80009F6780E870E060E008959FEF80EC0895C2
:107C900000240A94161617061806090608950024EB
:107CA0000A9412161306140605060895092E039465
:107CB000000C11F4882352F0BB0F40F4BF2B11F4D9
:107CC00060FF04C06F5F7F4F8F4F9F4F089557FD38
:107CD0009058440F551F59F05F3F71F04795880F3A
:107CE00097FB991F61F09F3F79F0879508951216D1
:107CF00013061406551FF2CF4695F1DF08C016167D
:107D000017061806991FF1CF86957105610508942D
:107D10000895E894BB2766277727CB0197F9089544
:107D20000BD0C4CFB5DF28F0BADF18F0952309F0E7
:107D3000A6CFABCF1124EECFCADFA0F3959FD1F32E
:107D4000950F50E0551F629FF001729FBB27F00D09
:107D5000B11D639FAA27F00DB11DAA1F649F66275E
:107D6000B00DA11D661F829F2227B00DA11D621FAD
:107D7000739FB00DA11D621F839FA00D611D221F67
:107D8000749F3327A00D611D231F849F600D211D4B
:107D9000822F762F6A2F11249F5750408AF0E1F0EE
:107DA00088234AF0EE0FFF1FBB1F661F771F881F37
:107DB00091505040A9F79E3F510570F060CFAACF77
:107DC0005F3FECF3983EDCF3869577956795B79522
:107DD000F795E7959F5FC1F7FE2B880F911D96954C
:107DE000879597F90895629FD001739FF001829F54
:107DF000E00DF11D649FE00DF11D929FF00D839F3A
:107E0000F00D749FF00D659FF00D9927729FB00DD6
:107E1000E11DF91F639FB00DE11DF91FBD01CF01E9
:107E200011240895991B79E004C0991F961708F052
:107E3000961B881F7A95C9F780950895AA1BBB1BCE
:107E400051E107C0AA1FBB1FA617B70710F0A61B5A
:107E5000B70B881F991F5A95A9F780959095BC017B
:107E6000CD01089597FB092E07260AD077FD04D08F
:107E7000E5DF06D000201AF4709561957F4F0895D4
:107E8000F6F7909581959F4F0895A1E21A2EAA1BAF
:107E9000BB1BFD010DC0AA1FBB1FEE1FFF1FA217BA
:107EA000B307E407F50720F0A21BB30BE40BF50BB7
:107EB000661F771F881F991F1A9469F76095709540
:107EC000809590959B01AC01BD01CF01089597FB72
:107ED000092E05260ED057FD04D0D7DF0AD0001C8E
:107EE00038F450954095309521953F4F4F4F5F4F57
:107EF0000895F6F790958095709561957F4F8F4F17
:107F00009F4F08952F923F924F925F926F927F9270
:107F10008F929F92AF92BF92CF92DF92EF92FF9299
:107F20000F931F93CF93DF93CDB7DEB7CA1BDB0B45
:107F30000FB6F894DEBF0FBECDBF09942A883988EA
:107F400048885F846E847D848C849B84AA84B984F1
:107F5000C884DF80EE80FD800C811B81AA81B981FD
:107F6000CE0FD11D0FB6F894DEBF0FBECDBFED0111
:107F70000895F999FECFB2BDA1BDF89A119600B44B
:107F80000895F7DF01921A94E1F70895F2DFE02DEA
:107F9000F0DFF02D0895F999FECFB2BDA1BD00BC70
:107FA00011960FB6F894FA9AF99A0FBE0895F3DF76
:107FB000012CF1DF112408950190EDDF1A94E1F70F
:047FC0000895FFCF52
:107FC4000AFF0164496E74656772616C4E69636B84
:107FD40020202020496E74656772616C526F6C6C4E
:107FE400202020204163634E69636B2020202020E1
:107FF40020202020416363526F6C6C2020202020BD
:10800400202020204779726F59617720202020207A
:108014002020202052656164696E6748656967683D
:10802400742020204163635A202020202020202017
:108034002020202047617320202020202020202081
:10804400202020205265636569766572204C657630
:10805400656C2020566F6C74616765202020202099
:10806400202020204D6F746F722046726F6E744C06
:10807400656674204D6F746F722046726F6E745211
:10808400696768744D6F746F7220526561724C65D4
:10809400667420204D6F746F72205265617252694C
:1080A400676874204D6F746F72205269676874201A
:1080B400202020204D6F746F72204C656674202040
:1080C400202020204163635F5A202020202020208C
:1080D40020202020535049204572726F72202020A6
:1080E40020202020535049204F6B20202020202086
:1080F400202020202020202020202020202020207C
:1081040020202020536572766F20202020202020FC
:10811400202020204E69636B202020202020202056
:1081240020202020526F6C6C202020202020202032
:10813400202020202020202020202020202020203B
:10814400202020202020202020202020202020202B
:10815400202020202020202020202020202020201B
:10816400202020202020202020202020202020200B
:1081740020202020202020202020202020202020FB
:1081840020202020202020202020202020202020EB
:1081940020202020202020202020202020202020DB
:1081A400202020204750535F4E69636B20202020FD
:1081B400202020204750535F526F6C6C20202020D9
:1081C40020202020FFFF010A6400007D0000FF033F
:1081D4000102030405060708090A48656C6C6F2050
:1081E400576F726C64000000000000000000000083
:1081F400000000000000000000000000000000007B
:10820400000000000000000000000000000000006A
:10821400000000000000000000000000000000005A
:10822400000000000000000000000B016400FFFFDC
:10823400FFFFF40190D0030090D00300ECFF17B7C8
:10824400D13830FB103A409696020A000000000034
:10825400000000644600006401426567696E6E6553
:108264007200004E6F726D616C000053706F727417
:1082740000000001020203030303040404040404D1
:10828400040405050505050505050505050505059C
:10829400050506060606060606060606060606067C
:1082A400060606060606060606060606060606066A
:1082B400060607070707070707070707070707074C
:1082C400070707070707070707070707070707073A
:1082D400070707070707070707070707070707072A
:1082E400070707070707070707070707070707071A
:1082F40007070808080808080808080808080808FC
:1083040008080808080808080808080808080808E9
:1083140008080808080808080808080808080808D9
:1083240008080808080808080808080808080808C9
:1083340008080808080808080808080808080808B9
:1083440008080808080808080808080808080808A9
:108354000808080808080808080808080808080899
:108364000808080808080808080808080808080889
:028374000808F7
:00000001FF
